:020000040800F2
:100000005897002025030008BD4E0008074B000844
:10001000B94E00081129000895560008000000009C
:10002000000000000000000000000000C34E0008B7
:100030007F2A000800000000C14E0008C54E0008DD
:100040003F0300083F0300083F0300083F03000888
:100050003F0300083F0300083F0300083F03000878
:100060003F0300083F0300083F0300083F03000868
:100070003F030008152900083F0300082529000850
:1000800035290008452900083F0300083F03000800
:100090003F0300083F0300083F0300083F03000838
:1000A0003F0300083F0300083F0300083F03000828
:1000B0003F0300083F0300083F0300083F03000818
:1000C0003F0300083F0300083F0300083F03000808
:1000D0003F03000875560008855600083F030008D6
:1000E0003F0300083F0300083F0300083F030008E8
:1000F0003F0300083F0300083F0300083F030008D8
:100100003F0300083F0300083F0300083F030008C7
:10011000C54F00083F0300083F0300083F030008E5
:100120003F0300083F030008552900083F0300086B
:100130003F0300083F0300083F0300083F03000897
:100140003F0300083F0300083F0300083F03000887
:100150003F0300083F030008652900083F0300082B
:100160003F0300083F0300083F0300083F03000867
:100170003F0300083F0300083F03000800000000A1
:100180003F0300083F03000800F002F800F0BAF84F
:100190000AA090E8000C82448344AAF10107DA45E2
:1001A00001D100F0AFF8AFF2090EBAE80F0013F07A
:1001B000010F18BFFB1A43F0010318479C6D0000A4
:1001C000BC6D00000A444FF0000C10F8013B13F026
:1001D000070408BF10F8014B1D1108BF10F8015BA0
:1001E000641E05D010F8016B641E01F8016BF9D193
:1001F00013F0080F1EBF10F8014BAD1C0C1B09D1EA
:100200006D1E58BF01F801CBFAD505E014F8016B5B
:1002100001F8016B6D1EF9D59142D6D370470000ED
:100220000023002400250026103A28BF78C1FBD8FF
:10023000520728BF30C148BF0B6070476E2900F0DD
:10024000DD83702900F04F85662906F0C485652995
:1002500006F0C185672906F0BE85612906F0BD85D7
:1002600003681B0A28BF41F08001692900F058810A
:10027000642900F05581752900F052816F2900F042
:10028000DC84782900F01B85E92900F07784E429D3
:1002900000F07484F52900F07184EF2900F0D9840E
:1002A000F82900F01A850368DB0928BF41F08001B6
:1002B000632900F0E683732900F0EB83E32901F062
:1002C0002B81F32901F03081002070471FB506F023
:1002D0007DFD9DE8030001F005FD01F049FA0400F1
:1002E0000020002106F05CFD401C60600020002121
:1002F00006F040FDE06001F01FF91FBD10B501F0F0
:1003000084F910BD01F007FA1146FFF7DFFF06F090
:1003100051FC01F0B5FC03B4FFF7F0FF03BC01F0A2
:1003200093FE00000948804709480047FEE7FEE7C2
:10033000FEE7FEE7FEE7FEE7FEE7FEE7FEE7FEE795
:1003400004480549054A064B70470000B14F0008B4
:1003500089010008589100205897002058930020E8
:100360005893002053EA020C00F069802DE9F04B0D
:100370004FF00006002B1FBFB3FA83F503FA05F414
:1003800024FA05F65E4012BF1643B2FA82F502FA6D
:1003900005F4C5F120051EBF22FA05FC44EA0C0451
:1003A000203556EA044C4FEA144418BF641C4FF041
:1003B00000084FF00009904271EB030C39D300297B
:1003C00019BFB1FA81F701FA07F6B0FA80F700FA1F
:1003D00007F6C7F120071EBF20FA07FC46EA0C0605
:1003E0002037B6FBF4FCA7EB0507103F07F01F0B07
:1003F000CBF120060CFA0BFB2CFA06F644BFB346F1
:100400000026202FA4BF5E464FF0000B5BEA060CCF
:1004100008BF4FF0010B19EB0B09ABFB027C48EB5B
:100420000608C01B06FB02CC0BFB03CC71EB0C01D6
:10043000C1E70B46024641464846BDE8F08B13B57E
:100440004FF000004FF00001AFF30080BDE81C400A
:10045000704700007CB51D4616460C00009001D088
:100460002044401E074B7B442A4669460190304693
:1004700000F0DDFA05461CB10020694600F0EAFAFA
:1004800028467CBDF50500000FB4044910B503AA49
:10049000029800F003FB10BC5DF814FB4C900020A8
:1004A0000FB41CB5084B06AA7B446946009005981A
:1004B00000F0BDFA04460020694600F0CBFA204661
:1004C0001CBC5DF814FB0000A905000070B50C46CB
:1004D0000546012A05D02878800600D5EA69002360
:1004E00002E0012305E05B1C934202D2E05C00289D
:1004F000F9D1A869E618C01AA861286A18442862C8
:10050000284600F0E9F904E0D5E9012114F8010BCF
:100510009047B442F8D3284600F0F4F970BD0000CB
:100520002DE9F0410646002410687529314616A5CC
:1005300010D000F0F8F9002802DA404213A507E0D5
:1005400031688A0701D512A502E0490704D511A533
:10055000012401E000F0F0F900210A2206F124074D
:1005600009E0B0FBF2FCB0FBF2F302FB1C00303000
:1005700078541846491C0028F3D123462A463046B1
:10058000BDE8F04100F0E1B9000000002D000000DE
:100590002B000000200000002DE9F05F8946044692
:1005A0004FF0000ADFF874B1FB44C0F820A02046E9
:1005B000E1688847002874D0252806D0D4E90121B5
:1005C0009047206A401C2062F1E700265F462046E3
:1005D000E16888472028054607DB312D05D27819C8
:1005E00010F8200C08B10643F1E7B00701D526F05A
:1005F0000406C4F81CA00027C4F818A02A2D09D0AE
:10060000284605F07DF838B304EB8708303DC8F87C
:10061000185019E059F8041B204604EB8702916139
:10062000E1688847012F054618D1E069002820DAE3
:1006300026F020061DE0D8F8180000EB800005EB3E
:1006400040003038C8F818002046E1688847054661
:1006500005F056F80028EED1012F0AD02E2D08D132
:100660002046E16888477F1C0546022F46F0200699
:10067000C4DBA069002803DA404246F00106A0610D
:10068000F00701D026F010066C2D0BD0682D09D094
:100690004C2D39D06A2D35D0742D35D07A2D33D0EC
:1006A00016E038E0E1682F4620468847B842054604
:1006B00009D16C2F26D04FF48060E16806432046B4
:1006C0008847054604E06C2F1AD04FF4807006432B
:1006D0000DB3A5F14100192802D8203546F4006673
:1006E0004A462946204626604E46FFF7A7FD80B1C0
:1006F00001280BD0F61D26F0070000F1080956E787
:100700004020E4E78020D8E70020D6E706F104097E
:100710004DE7284652E7206ABDE8F09F5268000086
:1007200040EA010310B59B070FD1042A0DD310C86E
:1007300008C9121F9C42F8D020BA19BA884201D9C0
:10074000012010BD4FF0FF3010BD1AB1D30703D008
:10075000521C07E0002010BD10F8013B11F8014BBE
:100760001B1B07D110F8013B11F8014B1B1B01D1DA
:10077000921EF1D1184610BD10B5431C02E010F8CE
:10078000011B71B18107FAD14FF0013202C88C1AF6
:100790008C4314EAC211F9D0C01A0A0603D0C01E55
:1007A00010BDC01A10BD0A0401D0801E10BD090280
:1007B000FCD0401E10BD032A40F2308010F0030C24
:1007C00000F0158011F8013BBCF1020F624498BFA4
:1007D00011F801CB00F8013B38BF11F8013BA2F141
:1007E000040298BF00F801CB38BF00F8013B11F0BC
:1007F000030300F08382083AC0F0088051F8043BFC
:10080000083A51F804CBA0E80810F5E7121D5CBFC8
:1008100051F8043B40F8043BAFF30080D20724BFFB
:1008200011F8013B11F801CB48BF11F8012B24BF8F
:1008300000F8013B00F801CB48BF00F8012B7047DE
:100840004FF000020429C0F0128010F0030C00F0F9
:100850001B80CCF1040CBCF1020F18BF00F8012B77
:10086000A8BF20F8022BA1EB0C0100F00DB85FEA45
:10087000C17C24BF00F8012B00F8012B48BF00F811
:10088000012B70474FF0000200B513469446964680
:10089000203922BFA0E80C50A0E80C50B1F1200193
:1008A000BFF4F7AF090728BFA0E80C5048BF0CC041
:1008B0005DF804EB890028BF40F8042B08BF70479F
:1008C00048BF20F8022B11F0804F18BF00F8012B11
:1008D000704770477047704770B504468569006877
:1008E000C10601D5302600E02026C00707D070BD24
:1008F000D4E9012130469047206A401C20626D1ED9
:10090000F6D570BD70B5044685690078C00707D17B
:1009100070BDD4E9012120209047206A401C20624C
:100920006D1EF6D570BD09684A0501D540B2704705
:10093000C905FCD500B2704709684A0501D5C0B2A7
:100940007047C905FCD580B270472DE9F0470D46C8
:1009500099469246044600F124080168880604D5A9
:10096000E06921F01001216000E00120A84201DDD2
:10097000471B00E00027A1697A1902EB0900081A59
:10098000A0612078C00602D42046FFF7A5FF00260C
:1009900008E0D4E901211AF806009047206A401CBB
:1009A000761C20624E45F4DB2078C0060AD520462E
:1009B000FFF792FF06E0D4E9012130209047206A3A
:1009C000401C2062381EA7F10107F4DC07E0D4E9DF
:1009D000012118F805009047206A401C2062281E5B
:1009E000A5F10105F3DC2046FFF78CFF2078000617
:1009F00002D50220BDE8F0870120FBE711680268FC
:100A0000006A530501D508700AE0D30501D50880B6
:100A100006E0130603D5C217C1E9000200E0086032
:100A20000120704701694A1C02610878704700B5CF
:100A30008FB0CDE901310021059105497944CDE917
:100A4000031011466846FFF7A7FD0FB000BD000078
:100A5000E5FFFFFF0A6802F8010B0A607047D1E961
:100A600000239A4202D2531C0B601070704710B5DD
:100A7000436913B1AFF3008001E0FFF727FD0120C8
:100A800010BD127800F124010A7000224A70012280
:100A9000EDE711684FF0FF32E9E70000074B70B552
:100AA0000D467B44FFF7C3FF0446284600F040FD97
:100AB00010B14FF0FF3070BD204670BD1D520000D8
:100AC0002DE9FF5F15468A460446DFF8AC80F844FE
:100AD0000027D8E900103E46CDE9001010E03AF8B2
:100AE00016106A4602A800F0C3FD411C07D0217809
:100AF000890603D5E269391891420DD80744761C5E
:100B00002078800602D5E069B84205DDAE42E6DB1A
:100B10003AF816000028E2D1A069C01BA061204667
:100B2000FFF7DAFED8E90010CDE90010002017E049
:100B30003AF818106A4602A800F09AFDB0F1FF3F9B
:100B400081460BD000250DF1080B05E0D4E9012109
:100B50001BF8050090476D1C4D45F7D308F10100C7
:100B6000B0428046E4DB206A384420622046FFF72A
:100B7000C9FEBDE8FF9F00003E6300002DE9F04183
:100B80008046D21D22F007020025D2E90002F52995
:100B900015A614D0011E72F1000106DA0023D0EB75
:100BA000030063EB020211A608E0D8F800108B07DF
:100BB00001D50FA602E0490701D50EA60125114671
:100BC000002408F1240704E000F0CAF830323A5556
:100BD000641C50EA0102F7D12B46324621464046BA
:100BE000BDE8F041FFF7B1BE000000002D0000009D
:100BF0002B0000002000000030B4002100F124048C
:100C000008E002F00705D208303542EA4372DB08FB
:100C10006554491C52EA0305F3D10468002310A26D
:100C2000250707D5A40600D421B1C46901230DA26C
:100C3000641EC46130BCFFF788BE10B5044621466F
:100C40001068FFF779FE02462046BDE810400023F9
:100C5000D2E7D21D22F00701D1E90023CCE7000042
:100C60000000000030000000F0B40D4601880905C6
:100C700002D5214C7C4402E01F4C7C440E34002100
:100C800000F1240608E002F00F071209E75D42EACE
:100C900003721B097754491C52EA0307F3D1027807
:100CA0000023120704D5702D06D009B10223113498
:100CB0002246F0BCFFF749BE01231034F8E770B5B7
:100CC00004460D4621461068FFF736FE02462946C7
:100CD0002046BDE870400023C6E7D21D22F007037E
:100CE000D3E90023C0E70368126843F020030360E0
:100CF0000823C3610023B7E7A061000010B5203AC4
:100D0000C0F00B80B1E81850203AA0E81850B1E8C4
:100D10001850A0E81850BFF4F5AF5FEA027C24BF7A
:100D2000B1E81850A0E8185044BF18C918C0BDE871
:100D300010405FEA827C24BF51F8043B40F8043B3A
:100D400008BF7047D20728BF31F8023B48BF11F8EF
:100D5000012B28BF20F8023B48BF00F8012B704749
:100D600030B5B0F10A024FEA900E71F100034EEA7D
:100D7000817EB0EB0E0061EB91014FEA101E4EEA4E
:100D8000017E10EB0E0041EB11114FEA102E4EEADE
:100D9000016E10EB0E0041EB11214FEA104E4EEAAE
:100DA000014E10EB0E0041EB1141401841F10001E2
:100DB0004FEAD00040EA41704FEAD10110EB8005C4
:100DC0004FEA810444EA907444EB01046D1944EB4A
:100DD0000404521BA3414FF0000348BF0A3200D560
:100DE00030BD401C41F1000130BD70472DE9FF4F7F
:100DF0000C461E464FF0FF378BB0D2E90001DDF8FC
:100E000060800A908A46C1F30A5505B93D46002123
:100E100008464FF00000BAF1000F00F4400005DA78
:100E200000EB80004FF4400101EA50004FEA905976
:100E3000B9F1010F00DDB9460A9850EA4A000ED018
:100E400044F61050A5F2FF3545432F14B8F1000FBA
:100E50001ED07542291E1EDDC9F100021CE0B8F14A
:100E6000010F4FF0000001D0302103E0F24305E014
:100E70002154401CB042FBDB3046002200212154AB
:100E80000B99C1F80880C1E900200FB0BDE8F08FD0
:100E9000BD1B6D1CDEE74A4600DA694206A800F079
:100EA000D3FC06AB93E8070003AB83E8070050468A
:100EB0000A9901F065F98DE80700A0F500501F3888
:100EC00000900398002D0ADD42F21F014A460844B3
:100ED000002303A90390684601F0CEFB09E0A0F5CA
:100EE00000504A461F38002303A90390684601F0CA
:100EF000D8FB8DE807000004000C03D04FF0FF3052
:100F0000410800E01046B8F1000F03D00022009223
:100F100015461EE0751E05D4FFF722FF30326255DC
:100F20006D1EF9D5B3460122084302D000227F1C72
:100F300004E02078302801D100227F1E002A099782
:100F400084D01DE0112D07DAFFF70AFF3032625519
:100F50006D1C50EA0102F5D1084302D00098C8B1D7
:100F60000EE00021681E05E0235C625C635422549D
:100F7000401E491C8142F7DBAB46A81B401E09906E
:100F8000002004F80B000B98099AC0F80880C0E90B
:100F9000002B7AE711264FF0000857E72DE9F04FB4
:100FA00088460446D21D22F0070191B0D1E9000124
:100FB000CDE90A0104F070FB02460B98C00F01D086
:100FC0002D2007E02068810701D52B2002E0202199
:100FD00001EAC000032A099001D0072A05DB034675
:100FE0004146204600F0F0FB0BE12078800601D559
:100FF000E06900E00620B8F1650F814606D0B8F13F
:10100000660F18D0B8F1670F70D131E00020B9F148
:10101000110F009001DB112301E009F101030AAA7D
:1010200001A90CA8FFF7E2FEDDE90C70002609F12A
:101030000105834647E001204B4600904FF00047F2
:101040000AAA01A90CA8FFF7D1FEDDE90DB00C99A1
:101050005D46002610B909F101000D18B9EB050035
:1010600003D4C0F1FF3609F10105A5EB09002BE01F
:10107000B9F1010F01DA4FF001090020B9F1110FA8
:101080000090484601DD112300E003460AAA01A9A9
:101090000CA8FFF7ABFEDDE90C704D460026834639
:1010A000207800070AD4AB4500DA5D4601A8012D7F
:1010B00004DD411911F8011C302907D04F4502DA2F
:1010C00017F1040F04DA012082460FE06D1EEEE7EF
:1010D000002F02DCED1B3E4403E0781CA84200DD3B
:1010E0007D1CB81B00F1010A4FF000472078000773
:1010F00003D4AA4501DB4FF0FF3A0021B7F1004FBE
:101100000DF143088DF8431024D002202B23002F2B
:1011100001DA7F422D230A21021EA0F1010000DC2A
:101120005FB197FBF1FC97FBF1F201FB1C7C1746CA
:101130000CF1300C08F801CDEEE7A8F101000370C6
:101140002188090501D5452100E06521A0F10108AC
:1011500000F8011C09980FA9A1EB0807FF1D00B1B9
:101160000120411901EBEA70A1693844081A401EB8
:10117000A0612078C00602D42046FFF7ADFB099895
:1011800028B1D4E901219047206A401C20622078D0
:10119000C00622D52046FFF79FFB1EE0002E04DB91
:1011A000B34502DD01A8805D00E03020D4E90121D3
:1011B0009047206A401C2062761CAAF101005FEA79
:1011C000000A0AD100F0D4FAC0680168405CD4E992
:1011D00001219047206A401C2062281EA5F10105CC
:1011E000DCDC07E0D4E9012118F8010B9047206A04
:1011F000401C2062381EA7F10107F3DC2046FFF7F0
:1012000081FB032011B041E62DE9F04F04460D4665
:10121000D21D22F0070089B0D0E900974846394630
:1012200004F03AFA0246F80F01D02D2307E02068B7
:10123000810701D52B2302E0202101EAC0038DF8AC
:1012400020300BB1012000E00020032A824601D0AB
:10125000072A04DB2946204600F0B6FA3FE1207851
:10126000800601D40D2500E0E569C7F30A560D2D6F
:1012700049DA00214FEA175B08464FF00000002FC3
:1012800000F4400007DA00EB80004FF4400100EB6F
:10129000D07001EA60008115012901DD4FF0FF31B6
:1012A00000224FEA850CBCF1180F06D31346ACF1AF
:1012B00018004FF08052C24003E04FF4801323FA2D
:1012C0000CF30CF10C0CBCF1200F04D3ACF1200C8E
:1012D00009FA0CF001E007FA0CF000294FF0004881
:1012E00001DD18B90FE00ED140450CD319EB02090E
:1012F0005F4121B9404502D19F4329EA0209BBEB76
:10130000175F00D0761C2088000502D57B48784402
:1013100002E07A487844193808AA302302F80A30E3
:10132000037C0AF10101002E0AF1020A53546A46B5
:1013300002DC4FF0300101E04FF031014FF00108C5
:101340008DF8001002D0A6F2FF3603E059EA4701FB
:1013500000D06B4E002D02DC2178090704D54FF038
:1013600002082E218DF80110C44600210BE0C7F3BE
:1013700003433F01C35C491C6D1E02F80830052978
:1013800008F1010801DA002DF1DC00210CE000EB8E
:101390001973491C1B786D1E082902F808304FEAA2
:1013A000091908F1010801DA002DF0DC21688B062B
:1013B00002D516E0A8F10108E04505DD02EB0803BF
:1013C00013F8013C302BF5D0B8F1000F09DD02EB2A
:1013D000080313F8013C2E2B03D1090701D4A8F10F
:1013E0000108002D05DD3E2102F808106D1E08F1F0
:1013F0000108407C002E02F8080008F1010804DA18
:101400002D20764202F8080002E02B2002F80800A6
:101410000A214FF47A70864208F101080BDB96FB33
:10142000F0F3303302F8083096FBF0F308F10108CE
:1014300000FB136601E0642E0CDB642096FBF0F3E6
:10144000303302F8083096FBF0F308F1010800FB96
:10145000136601E00A2E06DB96FBF1F0303002F84D
:10146000080008F1010896FBF1F001FB1060303034
:1014700002F80800A16908F1010808EB050202EB77
:101480000A00081AA0612078C00602D42046FFF79F
:1014900023FA216A08AE01EB0A00206204E0D4E9D5
:1014A000012116F8010B9047BAF1010AF7D2207812
:1014B000C00602D52046FFF70FFA6E4609E016F87F
:1014C000010B3E280FD0D4E901219047206A401C2F
:1014D0002062B8F10108F2D22046FFF713FA09B0F2
:1014E0000320BDE8F08F206A2844206203E0D4E99D
:1014F0000121302090476D1EEBD3F8E7415B0000DF
:1015000002FCFFFF10B5436913B1AFF3008001E0A7
:10151000FFF7D6FA012010BD128800F12401828461
:101520000022C2840122EDE711684FF0FF32E9E7A3
:10153000007B00F08000704710B542485421FFF74F
:10154000A1F941485421FFF79DF940485421FFF784
:1015500099F93F493B483C4A3F4B08603D490A6086
:101560003A491960531C0365481C10650120086541
:101570003B48344A39A1784400F0E6FA20B93848AB
:1015800078440A3800F085FB37482F4A35A1784463
:1015900000F0DAFA20B9344878440A3800F079FBD0
:1015A00032482A4A2FA1784400F0CEFA20B92F48B9
:1015B00078440A3800F06DFB40232248DC0000210B
:1015C000224600F09EFA20B125487844543800F0B5
:1015D00060FB1D4822464023002100F092FA20B112
:1015E00021487844543800F054FB18482246102310
:1015F000002100F086FA002806D01C487844BDE897
:101600001040563800F045BB10BD104870B5006D55
:1016100020F001040B4800F00DFB0B4800F00AFB22
:101620000A4800F007FB09E0206D20F00105204684
:1016300000F000FB204600F09FF82C46002CF3D170
:1016400070BD0000F88F00204C900020A09000207A
:101650008C02002090020020940200207200000002
:10166000EC58000077000000D8580000C458000073
:1016700070B516460C46054600F072F8036893F8FC
:101680000101012806D0FF2C0FD8185D68B1012098
:101690002C7070BDD3F807013246214603F20713C0
:1016A00003442846BDE8704018474FF0FF3070BD36
:1016B0000EB5CDE90001FFF75FF802906946012001
:1016C000ABBE0EBD08B5694600900220ABBE08BD9A
:1016D0001FB58DE8070069460520ABBE04B010BDFC
:1016E0001FB58DE80F0069460620ABBEF6E708B5CA
:1016F000694600900920ABBE08BD1CB5CDE90001CC
:1017000069460A20ABBE1CBD704708B5694600900B
:101710000C20ABBE08BD754600F0C2FAAE4605000F
:101720006946534620F00700854618B020B5FEF7FD
:1017300007FEBDE820404FF000064FF000074FF0D5
:1017400000084FF0000B21F00701AC46ACE8C009DF
:10175000ACE8C009ACE8C009ACE8C0098D467047E8
:1017600010B500F005F8001D10BD00BF3556000093
:10177000004870471491002070B50446051F00F022
:1017800095FA0068002C14BF446870BD002C18BF87
:10179000AC423CBF20466468F8D301680A18AA42EC
:1017A00018BF456003D12A680546114401602868C6
:1017B0004119A1421CBF6C6070BD616869602168FD
:1017C0000844286070BD00002DE9F0411F46044622
:1017D00003260168072A01F4006004DB08B116A59E
:1017E00005E016A503E008B115A500E015A521F058
:1017F00010002060A069C01EA0610FB1401EA06152
:101800002046FFF769F84FB1D4E9012138469047E7
:10181000206A401C2062C01C206206E0206AFAE7B1
:10182000D4E9012115F8010B9047761EF8D2204625
:10183000FFF768F8BDE8F0814E414E006E616E0022
:10184000494E4600696E66002DE9F047814616460E
:101850008AB0354878440DC88DE80D003248784488
:10186000801C03AC0DC884E80D0041F69B30084491
:10187000372190FBF1F290FBF1F5A5F1800501FB1A
:1018800012041B3C02D56442012000E00020DFF876
:1018900098A080460027FA44AAF1BE0A0EE0E007AD
:1018A0000AD03246684607EB470101230AEB810163
:1018B00000F0F7FE8DE8070064107F1C002CEED1CD
:1018C000194F7F44AE3F19E0E80715D007EB04102D
:1018D0000DF1180A90E80E008AE80E00C068F04288
:1018E00001D1981908903246012306A903A800F0F7
:1018F000D8FE03AB83E807006D10641C002DE3D114
:101900004FF0010332466946B8F1000F03A802D038
:1019100000F0B2FE01E000F0C4FEC9E90001C9F820
:1019200008200AB0BDE8F087985600002DE9F0477E
:1019300005460C46C86820F4201040F48000C860BA
:10194000800602D5084600F0FEFAE06841F2820106
:101950004FF0FF390140022903D0204600F09CFAE5
:10196000B5E000F42041B1F5004F0FD1C00306D51A
:101970006168E06A884200D80846606006E0206935
:10198000E06260606069FFF7C0FEA061A0680022AD
:10199000EEB200280DDAE1688B050AD4C043A060DE
:1019A00041F490302260E0606068411C6160067024
:1019B000A5E0E0689046226040F40050E0602069B5
:1019C00068BB6069FFF793FE012704F12405A0B10D
:1019D000A08910F4407F08D0E06900F0B2F92061DE
:1019E00018B1E06840F4006016E0E7612561E06846
:1019F00020F4407040F480600EE0E06900F0A1F94E
:101A000000282061F1D0E06840F4006010F4407FCD
:101A1000E06002D140F48070E06020696060E068BE
:101A200025696FF0010AC1051FD56168E06A884227
:101A300000D80846411B04D02246284600F036FA5A
:101A4000F0BBE068010203D5E562C4E9015854E047
:101A5000691CE1626160E16940F48030491EC4E9BB
:101A6000021030462E70BDE8F087010202D500F466
:101A700080320AE06068411C61600670E0680A2EEE
:101A800040F48030E06006D00022E16A6068814264
:101A900003D90B4602E00122F7E70346A7895B1B47
:101AA0007F0503D4E7699F4200DDE2B1814200D89F
:101AB0000146E5620F1AC4E90158002B09DD00E078
:101AC00005E022461946284600F0F0F908B14846DC
:101AD000C9E747B1A069E5626560C01BA061E06825
:101AE00040F01000E060E068000208D56168A0697D
:101AF000E562491B08446560A0615046B3E7304683
:101B0000B1E770B5C468A50713D0650211D4B2F56A
:101B1000807F09D0B2F5007F06D0B2F5806F08D182
:101B2000012300F1240106E05D1E6FF07F46B542FF
:101B300001D3012070BD0161C361416024F4706173
:101B40001143C160002070BD2DE9F0410C460746ED
:101B50001646104600F06EF82078611C61280AD005
:101B6000722802D077283CD102E00125002405E04C
:101B70000225042402E0082448F2020511F8010BB2
:101B80002B2806D0622809D011F8010C74280AD03D
:101B90000BE045F0030544F00204EFE745F00405CF
:101BA00044F00104EAE744F0100438462146FFF708
:101BB0007FFD411C15D00021316171604FF400712F
:101BC000F560F1617061200704D5304602220021E2
:101BD00000F0E6F8306D40F0010030653046BDE8B9
:101BE000F0810020FBE72DE9F0410D460646104C40
:101BF000206DC10704D0410804D020F00104F7E7AC
:101C000022460EE0542000F09CF807000ED0206D14
:101C100047F001010843542120653846FEF732FEA3
:101C20003A4629463046BDE8F0418DE70020D6E728
:101C3000F88F00202DE9F04704464FF000094FF0DF
:101C4000FF37C568D4E90486A80707D0204600F00E
:101C500057F93046FFF736FD002802DA3846BDE86E
:101C6000F087280502D54046FFF786FD4C21204627
:101C7000FEF708FE206D20F0010020654846EEE7E3
:101C800010B50446AFF300802046BDE81040FEF7D3
:101C900042BB10B500F07EF9BDE8104000F074B909
:101CA00000487047F49000207047000000487047DB
:101CB000FC900020704770477047704738B5044665
:101CC0000A4600206946AFF30080002808BF38BDEF
:101CD00002460099204600F0C4F9012038BD0120D9
:101CE00000F013BAF8B5AFF30080054600200C46AB
:101CF000102000BF0646A819A0420DD932466946F9
:101D00000020AFF30080070008BF00F0FEF9009844
:101D1000A04218BF0546C419FFF7C8FF0560074673
:101D2000F01D20F007004619284600F093F9B44250
:101D300008BFF8BDA21B31463868BDE8F84000F086
:101D400090B970B50646FFF7B1FF056806F10B00C4
:101D500020F00704B4429CBF002070BD2B466A6887
:101D6000BAB11068A04210D304F1080188423CBF08
:101D70005068586007D35168101941601168091BF9
:101D8000016058601460101D70BD13465268002A2F
:101D9000E7D121462846FFF791FF0028DED170BD2C
:101DA0002DE9F041044616460D464769007B800741
:101DB0002ED03846FFF79BFC50BB3EB3012E02D01D
:101DC000022E25D104E0204600F065F905441DE00F
:101DD0003846FFF79AFCE168002841F01001E16005
:101DE00005DA204600F058F80120BDE8F081C9036B
:101DF0000BD56268E16A914200D81146A26911448C
:101E00002269891A814200DD08460544002D01DA65
:101E10000220EAE7E16A6068E268814206D2910343
:101E2000E06203D522F4003141F01002A6690027D8
:101E3000AE4213DCE16A814201D90B4600E0034661
:101E400003EB060C2369ACEB030CAC4506DD8142C9
:101E500001D98C4600E084469C4505D1A7602760E7
:101E600042F02000A5620DE0AD1BE669AE1B814289
:101E7000A66000D90846C01A281A20605819606068
:101E800022F0200003490840E060002084F84870F8
:101E9000ABE70000BFCFD7FFC16821F4001141F0CC
:101EA0008001C16000218160016070472DE9F04729
:101EB000814614460E464FF0FF383248D5685769C0
:101EC000054209D03846A169FFF717FC002811DB4D
:101ED0002C48C0430540E5602B463246494638460B
:101EE000FFF7F6FBA16920F00042B21A1144002866
:101EF000A16103D02046FFF7CFFF4046BDE8F08741
:101F000070B504460569C06A6168884200D8084611
:101F1000E16821F42011E160C90312D5A84208D07C
:101F20002246411B2846FFF7C1FF10B14FF0FF309A
:101F300070BD0020E562C4E90150E06820F4803003
:101F4000E060002070BD10B50446C06820F020009D
:101F5000E060A16AA06988420DD02046FFF7D0FF5B
:101F6000E06820F4405040F01000E060A06AA061FA
:101F70002069E062606044F24001E0688843E0600C
:101F800010BD000010000200002801D000F05CB875
:101F90007047000010B5014602A000F09DF8012036
:101FA00010BD000053494752545245443A205265EF
:101FB0006469726563743A2063616E2774206F7080
:101FC000656E3A20000000004FF0013C50F8042BF1
:101FD00051F8043B9A4221D1A2EB0C03934313EA3C
:101FE000CC1317D150F8042B51F8043B9A4215D169
:101FF000A2EB0C03934313EACC130BD150F8042B40
:1020000051F8043B9A4209D1A2EB0C03934313EA23
:10201000CC13DBD04FF00000704700BFD01A01BADC
:10202000B1FA81F101F0180122FA01F0CB40C1F1BF
:102030002001DBB2C0B2C01A2CFA01F3D11A9143CD
:1020400011EAC311E6D1704701491820ABBEFEE783
:102050002600020000210160C0E901107047102035
:102060007047034640688C46002818BF88423CBF32
:1020700003464068F8D318681844884207D00CF12A
:10208000030020F00700001D411A521A0146081DE6
:102090000A60FFF771BB10B50146C268900703D014
:1020A000900607D5886A0AE000F03EF80121016039
:1020B000881E10BD8B69486818440B69C01A91F8D6
:1020C00048301BB191F84910401A10BD1103FCD5DE
:1020D0000028FADD401E10BD70B505460C460A20EA
:1020E00000E06D1C00F018F835B128780028F8D110
:1020F00002E0641C00F010F814B120780028F8D138
:10210000BDE870400A2000F007B810B500F010F8E4
:10211000BDE81040FFF738BF08B569468DF80000EC
:102120000320ABBE08BD000000487047F4900020BB
:1021300010B5012805D0002103A0FFF7CDFF012035
:1021400010BD09A1F8E7000053494752544D454DD1
:102150003A204F7574206F662068656170206D6548
:102160006D6F7279000000003A2048656170206D43
:10217000656D6F727920636F72727570746564003B
:102180005FEA400C08BF91F0000F4FEA8C234FEA42
:10219000C12243EA51514FEA1C5018BF00F5F040EC
:1021A0004FEA300018BF41F000415FEA6C5C00F07C
:1021B0002980BCF1FF3F08BF40F080407047130CFE
:1021C00006BF12044FF0100C4FF0000C130E04BFAA
:1021D00012020CF1080C130F04BF12010CF1040CD5
:1021E000930F04BF92000CF1020CD30F04BF5200F6
:1021F0000CF1010C11464FF00002A0F11F00A0EB02
:102200000C00704711F0004F08BF704731F00041DB
:102210003FF4D5AF0B0C06BF09044FF0100C4FF084
:10222000000C0B0E04BF09020CF1080C0B0F04BFCD
:1022300009010CF1040C8B0F04BF89000CF1020C96
:10224000CB0F04BF49000CF1010CCCF12003A0EB33
:102250000C0022FA03F302FA0CF241EA030100F146
:102260000100704720F07F4C80EA030023F07F4795
:10227000ACEB070303F57C5300F0004003F1FF03D0
:102280002DE980494FEA154B09B44FEA144325EA7A
:102290000B4E24EA03480FF2042606EB13274908E5
:1022A0003E785FEA320203FB0667C7F5000707FBCB
:1022B00006F64FEA54374FEAD64606F1020607FB08
:1022C000066CCCF1005C4FEA1C472CEA074C07FB7C
:1022D00006F40CFB06F504EB15464FEA961634BFE0
:1022E00000204FF000404FEAD13706FB07FC4FEAD1
:1022F0001C4C0CFB0BF7D21B03FB0CF761EB07012B
:102300000CFB0EF7B0EB074072EB17420CFB08F723
:1023100034BFA2EB0742B2EB074261EB17414FEA31
:102320000C444FEA910706FB07FC4FEA1C4C0CFBE0
:102330000BF7B0EBC74072EB573203FB0CF734BF1F
:10234000A2EBC742B2EBC74261EB57310CFB0EF771
:10235000B0EBC70072EB57720CFB08F734BFA2EB6F
:10236000C702B2EBC70261EB5771039F4FEA81616D
:1023700041EA921104EBCC044FEAD1374FEA826272
:1023800006FB07FC42EA90124FEA80604FEA1C4CC1
:102390000CFB0BF7D21B03FB0CF761EB07010CFBEB
:1023A0000EF7B0EB074072EB17420CFB08F734BF97
:1023B000A2EB0742B2EB074261EB17414FEA8C55A3
:1023C0004FEA910704EB9C2406FB07FC4FEA1C4CE8
:1023D0000CFB0BF7B0EBC74072EB573203FB0CF76B
:1023E00034BFA2EBC742B2EBC74261EB57310CFBE3
:1023F0000EF7B0EBC70072EB57720CFB08F734BF57
:10240000A2EBC702B2EBC70261EB577115EB4C258B
:102410004FEA816141EA92114FEA82624FEAD13775
:1024200042EA901206FB07FC44F100044FEA806088
:102430004FEA1C4C0CFB0BF7D21B03FB0CF761EBB8
:1024400007010CFB0EF7B0EB074072EB17420CFBD9
:1024500008F734BFA2EB0742B2EB074261EB17412A
:1024600015EB1C154FEA813141EA92414FEA823265
:1024700042EA90424FEA80304FEA0C7644F1000481
:1024800048EA03434EEA0B484FF0000EB2EB080C4B
:1024900071EB030724BF624639464EEB0E0E4FF038
:1024A000000B0018524149414BEB0B0BB2EB080CEF
:1024B00071EB03077BF1000B24BF624639464EEBFC
:1024C0000E0E4FF0000B0018524149414BEB0B0B25
:1024D000B2EB080C71EB03077BF1000B24BF6246E3
:1024E00039464EEB0E0E51EA020718BF46F00106C0
:1024F00016EB0E7655F1000254F1000103D5BDE84C
:102500008901BDE80088BDE88901BDE80048B61929
:10251000524141EB0101A3F10103704780807F7EAE
:102520007D7C7B7A79787776767574737271717049
:102530006F6E6E6D6C6C6B6A6A69686867666665FB
:102540006464636362616160605F5F5E5E5D5D5C89
:102550005C5B5B5A5A5959585857575656555555FA
:102560005454535352525251515050504F4F4F4E5A
:102570004E4D4D4D4C4C4C4B4B4B4A4A4A494949A8
:1025800048484847474747464646454545444444EA
:10259000444343434342424242414141002B9C4613
:1025A00030D477002BD01CB54FEA370703B44FF077
:1025B00010004FF01001BAF1000F06D0BCF1000F6F
:1025C000DCBF40F0080040F008014FF000000FBCF5
:1025D000BDE810400BF1010BBBF1010F08BF5FEA32
:1025E000170722BF12F1010211F101014FF0004162
:1025F00043F1000300F0004043EA00007047F9D3C4
:102600005708D0E746EA064613F1400F4FEA164650
:102610001FDD13F1200FDFBF16430A4600212033D0
:102620005B42BED0C3F1200746EA064602FA07F72E
:102630004FEA164646EA0706C3F1200722FA03F2DC
:1026400001FA07F721FA03F14FF0000342EA07020B
:10265000A7E746EA020646EA06464FEA164646EA73
:102660000106BCBF46EA0646360C4FF000034FF0A9
:1026700000024FF0000194E72DE9804C9A46934602
:1026800070B491E8380007C831EA400C48BF34EA1A
:10269000430C03D5FFF7E6FDFFF780FFF0BCBDE874
:1026A000008C2DE9804C9A46934670B491E838002E
:1026B00007C810F0804F08BF13F0804F03D100F01F
:1026C00005F8FFF76BFFF0BCBDE8008C20F07F47FA
:1026D00080EA030023F07F4C07EB0C03A3F57C5347
:1026E00000F00040A3F1FE0392F0000F00F0B38071
:1026F00095F0000F00F077802DE901494FEA114075
:102700004FEA144621EA004800FB06FC24EA06478B
:1027100008FB06F607FB08F800FB07F718EB06486E
:102720004CEB164C4FEA124B18EB07484FEA154694
:102730004CEB174022EA0B4E0BFB06FC25EA064742
:102740000EFB06F607FB0EFE0BFB07F71EEB064E15
:102750004CEB164C4FF000061EEB074E4CEB174BA4
:1027600018EB0B0840F1000018EB0E0B58EB0008BB
:1027700040F100008F1A4FF000013CBFC943661BB7
:1027800014BFB5EB040C00213CBFC943F61B4FEA54
:1027900017444EEA8E0E27EA04454FEA1C4704FB15
:1027A00007622CEA074C05FB07F70CFB05F604FB58
:1027B0000CFC16EB074642EB174216EB0C4642EBBD
:1027C0001C421BEB060658EB0202414146EA9E06FC
:1027D00001D5BDE80189B619524141EB0101A3F1D0
:1027E0000103BDE801894FEA14454FEA114724EA85
:1027F000054621EA074C05FB07F406FB07F70CFB2F
:1028000006F105FB0CFC11EB074144EB17444FEAC2
:10281000124711EB0C4144EB1C4422EA074C05FB28
:1028200007F206FB07F70CFB06F605FB0CFC16EBA4
:10283000074642EB174216EB0C4642EB1C456A1862
:1028400054F1000148BF7047B619524141EB0101F4
:10285000A3F10103704795F0000F37D04FEA114202
:102860004FEA144721EA024624EA074C02FB07F12B
:1028700006FB07F70CFB06F402FB0CFC14EB074409
:1028800041EB17414FEA154714EB0C4441EB1C4157
:1028900025EA074C02FB07F506FB07F70CFB06F6DB
:1028A00002FB0CFC16EB074645EB174516EB0C46F6
:1028B00045EB1C42121951F1000148BF7047B6198F
:1028C000524141EB0101A3F1010370474FEA144566
:1028D0004FEA114724EA054621EA074C05FB07F1B8
:1028E00006FB07F70CFB06F24FF0000605FB0CFC9D
:1028F00012EB074241EB174112EB0C4251EB1C412A
:1029000048BF7047921841EB0101A3F101037047E2
:1029100000BFFEE710B5024800F078FA10BD0000D5
:102920009C04002010B5024800F070FA10BD0000B1
:10293000FC04002010B5024800F068FA10BD000049
:102940001C06002010B5024800F060FA10BD00001F
:102950007C06002010B5024800F058FA10BD0000B7
:102960005C05002010B5024800F050FA10BD0000D0
:10297000BC0500200146087810381823B0FBF3F29C
:102980000848805CC865032A05D908686FF3090008
:10299000001D886503E008686FF309008865886D8D
:1029A00070470000DE6D0008014600208A6A8B69CE
:1029B000CBB932B1012A0DD0022A03D0032A10D19B
:1029C0000EE000BFCB6A03F08073B3F1807F00D1CB
:1029D000012007E0CB6AB3F1C07F00D1012001E004
:1029E00000E000BF34E08B69B3F5005F1AD132B16B
:1029F000012A07D0022A03D0032A11D10AE000BF1E
:102A000001200EE0CB6A03F08073B3F1807F00D128
:102A1000012006E0CB6AB3F1C07F00D1012000E0C5
:102A200000BF15E032B1012A05D0022A04D0032AE2
:102A30000CD103E000BF00BF012008E0CB6A03F027
:102A40008073B3F1807F00D1012000E000BF00BFA0
:102A5000704730B50468246824F4802405682C602D
:102A6000046863608468402C04D10468A260046830
:102A7000E16003E00468A1600468E26030BD704773
:102A800072B600BFFEE7000010B5002201B909E0F0
:102A9000012901D10A0205E0022901D10A0201E05F
:102AA0004FF440720E4B1B6823F440730C4C2360B0
:102AB00023461B681343236023461B6823F0F80357
:102AC000236023461B68022444EAC0042343044CC9
:102AD000236023461B6843F48033236010BD00004D
:102AE000103C02401C48006800F40070B0B11A4865
:102AF000006820F400701849086000BF08460068AC
:102B000040F4006008600846006820F40060086037
:102B100000BF0846006840F4007008600E48006876
:102B200000F48060B0B10C48006820F480600A496D
:102B3000086000BF0846006840F4805008600846FE
:102B4000006820F48050086000BF0846006840F428
:102B50008060086070470000003C02400A4A12682A
:102B600022F44072084B1A601A46126842F00402BE
:102B70001A601A4612684FF4803343EA00231A435E
:102B8000014B1A6070470000103C0240074A12686F
:102B900022F44072054B1A601A4612681A601A46EF
:102BA000126842F001021A6001707047103C024046
:102BB00010B50D49096821F440710B4C2160214684
:102BC000096841F4407121602146096841F0010122
:102BD0002160026000BF00BF00BFBFF36F8F00BF66
:102BE00000BF00BF436010BD103C0240084A12689D
:102BF00022F44072064B1A601A46126842F4807240
:102C00001A601A46126842F001021A600180704789
:102C1000103C0240084A126822F44072064B1A60C7
:102C20001A46126842F400721A601A46126842F09C
:102C300001021A6001607047103C0240234800689E
:102C400000F0100040B12248C06940F01000204957
:102C5000C86110201D4908601C48006800F0200071
:102C600040B11B48C06940F008001949C8612020E4
:102C7000164908601548006800F0400040B114484B
:102C8000C06940F004001249C86140200F49086043
:102C90000E48006800F0800040B10D48C06940F067
:102CA00002000B49C8618020084908600748006895
:102CB00000F0020040B10648C06940F0200004491D
:102CC000C861022001490860704700000C3C0240C6
:102CD000DC06002070B50446002500201449C861B8
:102CE00000F04EFC054609E0601C38B124B100F04C
:102CF00047FC401BA04201D9032070BD0D4800686D
:102D000000F480300028EFD10A48006800F001008C
:102D100010B10120074908600648006800F0F20081
:102D200018B1FFF78BFF0120E7E70020E5E700007F
:102D3000DC0600200C3C024070B50446A56D00F096
:102D40001FFC064694F83500022808D080206065F4
:102D500000BF002084F8340000BF012070BD20684F
:102D6000006820F01600216808602068406920F0A3
:102D7000800021684861206C08B9A06C28B12068E7
:102D8000006820F00800216808602068006820F0D2
:102D900001002168086010E000F0F2FB801B0528AC
:102DA0000BD920206065032084F8350000BF002087
:102DB00084F8340000BF0320D0E72068006800F0EA
:102DC00001000028E8D194F85C103F208840A860FA
:102DD000012084F8350000BF002084F8340000BFD3
:102DE00000BFBBE7014691F83500022803D08020E0
:102DF000486501207047052081F8350008680068A3
:102E000020F001000A6810600020F3E7F8B50446DE
:102E1000002000908C4800684FF41651B0FBF1F789
:102E2000A56D2E6894F85C1008208840304098B159
:102E30002068006800F0040070B12068006820F08D
:102E400004002168086094F85C1008208840A8609D
:102E5000606D40F00100606594F85C1001208840CE
:102E6000304068B12068406900F0800040B194F8BB
:102E70005C1001208840A860606D40F00200606531
:102E800094F85C1004208840304068B120680068E5
:102E900000F0020040B194F85C1004208840A86063
:102EA000606D40F00400606594F85C10102088406C
:102EB000304078B32068006800F0080050B394F800
:102EC0005C1010208840A8602068006800F4802012
:102ED00080B12068006800F4002028B9206CC8B1D7
:102EE0002046216C884715E0A06C98B12046A16C63
:102EF00088470FE02068006800F4807028B92068D7
:102F0000006820F0080021680860206C10B120469D
:102F1000216C884794F85C102020884030400028BD
:102F200065D02068006800F0100000285FD094F899
:102F30005C1020208840A86094F83500052828D12E
:102F40002068006820F01600216808602068406949
:102F500020F0800021684861206C08B9A06C28B17D
:102F60002068006820F008002168086094F85C1070
:102F70003F208840A860012084F8350000BF002071
:102F800084F8340000BF206D10B12046216D8847C1
:102F9000F8BD2068006800F4802080B120680068D7
:102FA00000F4002028B9606C10B12046616C88479D
:102FB0001DE0E06BD8B12046E16B884717E0206840
:102FC000006800F4807068B92068006820F0100084
:102FD00021680860012084F8350000BF002084F8D3
:102FE000340000BFE06B10B12046E16B8847606D94
:102FF00038B3606D00F00100F0B1052084F83500B1
:103000002068006820F001002168086000BF009877
:10301000401C0090B84200D905E02068006800F02C
:1030200001000028F3D100BF012084F8350000BF63
:10303000002084F8340000BFE06C10B12046E16C41
:10304000884700BFA4E700000C0000202DE9F041F4
:103050000446002500F094FA074614B90120BDE8A3
:10306000F081606A00B100BF022084F8350000BF23
:10307000002084F8340000BF2068006820F00100C0
:10308000216808600AE000F07BFAC01B052805D91A
:1030900020206065032084F83500E0E720680068A0
:1030A00000F001000028EED12068056821480540A5
:1030B000D4E901010843E1680843216908436169D3
:1030C0000843A1690843E1690843216A08430543AD
:1030D000606A042803D1D4E90B0108430543206842
:1030E00005602068456925F00705606A0543606A48
:1030F00004280DD1A06A0543E06A48B12046FFF7D5
:1031000053FC28B140206065012084F83500A6E713
:10311000206845612046FFF72DFC064694F85C10B8
:103120003F208840B06000206065012084F83500B1
:10313000002094E73F8010F02DE9F04704460D464B
:1031400016461F464FF00008D4F8589000BF94F878
:103150003400012802D10220BDE8F087012084F864
:10316000340000BF94F83500012825D1022084F8EE
:103170003500002060653B46324629462046FFF771
:1031800068FC94F85C103F208840C9F8080020686B
:10319000006840F0160021680860206C28B12068A3
:1031A000006840F00800216808602068006840F06E
:1031B00001002168086006E000BF002084F83400A8
:1031C00000BF4FF002084046C6E7000070B5044655
:1031D00000F0D6F906462546681C10B10448007870
:1031E000054400BF00F0CCF9801BA842FAD370BDA3
:1031F000080000202DE9F04104460E460127002575
:1032000000BF2548007E012802D10220BDE8F081E0
:1032100001202149087600BF4CF25030FFF75AFDDB
:103220000746002F31D1401E3060206801280FD1A1
:10323000207C6168FFF792FC4CF25030FFF74AFDAA
:1032400007461648006820F00400144908601AE098
:10325000A56812E0217C2846FFF716FC4CF250309E
:10326000FFF738FD07460D48006820F0FA000B49CB
:1032700008600FB1356005E06D1CD4E90210084408
:10328000A842E7D800BFFFF72DFC00BF002002498D
:10329000087600BF3846B9E7DC060020103C024043
:1032A0000348006840F00040014908600020704772
:1032B000103C02402DE9F04106460F4614461D46DB
:1032C0004FF0010800BF1F48007E012802D10220F4
:1032D000BDE8F08101201B49087600BF4CF2503058
:1032E000FFF7F8FC8046B8F1000F23D126B9E1B210
:1032F0003846FFF74BFC12E0012E04D1A1B238464C
:10330000FFF774FC0BE0022E04D121463846FFF78C
:1033100081FC04E022462B463846FFF749FC4CF27C
:103320005030FFF7D7FC80460748006820F00100C6
:103330000549086000BF00200249087600BF4046EA
:10334000C6E70000DC060020103C024000200949CE
:10335000096801F0004159B10749064A0C3A116069
:10336000064911600349096801F0004101B10120DB
:1033700070470000103C024023016745AB89EFCD48
:10338000F8B502460B460025002400200021D6E0B7
:10339000012606FA01F51E6806EA0504AC4274D15E
:1033A0001E7906F00306012E04D01E7906F00306EE
:1033B000022E13D190684F000326BE40B0434F0049
:1033C000DE68BE4030439060506801268E40B043B6
:1033D0001E79C6F300168E40304350601E7906F009
:1033E0000306032E09D0D0684F000326BE40B04329
:1033F0004F009E68BE403043D0601E7906F0030641
:10340000022E13D1CF0802F1200656F827004E07EE
:10341000F70E0F26BE40B0434F07FF0E1E69BE4099
:103420003043CF0802F1200646F8270010684F000D
:103430000326BE40B0431E7906F003064F00BE408F
:10344000304310605E6806F44036002E76D000BF30
:10345000002600963C4E366846F480463A4F3E6061
:103460003E46366806F48046009600BF00BF374EE1
:103470008F0856F827008E07370F0F26BE40B0433F
:10348000334EB24202D1002624E057E0314EB24220
:1034900001D101261EE0304EB24201D1022619E0D0
:1034A0002E4EB24201D1032614E02D4EB24201D17C
:1034B00004260FE02B4EB24201D105260AE02A4E27
:1034C000B24201D1062605E0284EB24201D10726BC
:1034D00000E008268F073F0FBE4030431B4E8F0889
:1034E00046F82700224E3068A0435E6806F4801636
:1034F00006B120431E4E3060361D3068A0435E6822
:1035000006F4001606B12043194E361D3060184EE1
:10351000361F3068A0435E6806F4003606B12043CB
:10352000134E361F3060361F3068A0435E6806F4C5
:10353000803606B120430E4E083E3060491C1029EB
:10354000FFF426AFF8BD00004438024008380140BF
:10355000000002400004024000080240000C02404B
:10356000001002400014024000180240001C0240FB
:10357000083C01400AB1816101E00B04836170479E
:103580000148006870470000000000200348006800
:103590000349097808440149086070470000002089
:1035A0000800002010B50D48006840F400700B4979
:1035B00008600846006840F48060086008460068BB
:1035C00040F480700860032000F0A6F8032000F0AB
:1035D00007F800F02BF8002010BD0000003C02406E
:1035E00070B504460E4800784FF47A71B1FBF0F0E4
:1035F0000C490968B1FBF0F5284600F013FD08B14D
:10360000012070BD102C07D200222146501E00F070
:1036100045F80548046001E00120F2E70020F0E7EA
:10362000080000200C0000200400002008B500BFA6
:10363000002000901048006840F480400E49086067
:103640000846006800F48040009000BF00BF00BF43
:1036500000200090081F006840F08050091F08609B
:103660000846006800F08050009000BF00BF0520B1
:1036700000F052F808BD00004438024001460846F8
:10368000002809DB00F01F0301229A4043099B0038
:1036900003F1E023C3F8002100BF70472DE9F05F7C
:1036A00080460D461646002702F00EF807463946BA
:1036B0002A46334601F00700C0F1070ABAF1040FA9
:1036C00002D94FF0040A01E0C0F1070AD14600F127
:1036D000040ABAF1070F02D24FF0000A01E0A0F18C
:1036E000030AD4464FF0010A0AFA09FAAAF1010ABC
:1036F0000AEA020A0AFA0CFA4FF0010B0BFA0CFB69
:10370000ABF1010B0BEA030B4AEA0B0421464046DE
:1037100001F0E2FFBDE8F09F00BF00F00702064B9A
:1037200019684FF6FF031940044B0B4343EA02218B
:10373000014B196000BF70470CED00E00000FA0576
:1037400070B504460D460CB9012070BD584800689C
:1037500000F00700A84209D255490D7008460068DC
:1037600000F00700A84201D00120EEE7207800F029
:10377000020002281DD1207800F00400042805D1A1
:103780004C48006840F4E0504A490860207800F056
:103790000800082805D14748006840F460404549C2
:1037A00008604448006820F0F000A16808434149DF
:1037B0000860207800F00100A8B36068012807D1F4
:1037C0003C4808380068C0F34040B8B90120BCE765
:1037D0006068022802D06068032807D1354808389D
:1037E0000068C0F3406048B90120AEE731480838AE
:1037F0000068C0F3400008B90120A6E72D48006822
:1038000020F00300616808432A490860FFF7B8FE0A
:10381000064609E0FFF7B4FE801B41F2883188427A
:1038200002D9032091E707E02248006800F00C006D
:103830006168B0EB810FEDD11D48006800F0070012
:10384000A84209D91A490D700846006800F007001F
:10385000A84201D0012078E7207800F00400042875
:1038600007D11448006820F4E050E168084311498A
:103870000860207800F00800082808D10D4800688A
:1038800020F46040216940EAC1000A49086000F064
:103890003FF808490968C1F30311074A515CC84061
:1038A0000649086006480068FFF79AFE00204CE7CA
:1038B000003C024008380240E66D00080C00002081
:1038C0000400002001480068704700000C00002040
:1038D00000B5FFF7F7FF04490968C1F38221034AE5
:1038E000515CC84000BD000008380240F66D000879
:1038F00000B5FFF7E7FF04490968C1F34231034A05
:10390000515CC84000BD000008380240F66D000858
:103910002DE9F047002400250026A146254800682F
:1039200000F00C0020B1042805D008283AD105E0A9
:10393000DFF8849039E0DFF8849036E01D48001FFE
:10394000006800F03F041B48001F006800F480007E
:1039500078B11A481749091F0968C1F38811A0FBFB
:1039600001700146224600233846FCF7FBFC054661
:103970000EE011480F49091F0968C1F38811A0FB27
:1039800001700146224600233846FCF7EBFC054651
:103990000848001F0068C0F30140401C4600B5FB0A
:1039A000F6F902E0DFF8109000BF00BF4846BDE81E
:1039B000F0870000083802400024F40000127A006A
:1039C000F8B504460CB90120F8BD207800F00100DC
:1039D000002874D0F948006800F00C0004280DD0CD
:1039E000F648006800F00C00082813D1F348001FC7
:1039F000006800F48000B0F5800F0BD1EF48083864
:103A00000068C0F34040002859D06068002856D1B3
:103A10000120D9E700BF6068B0F5803F08D1E748D2
:103A20000838006840F48030E449083908601EE036
:103A30006068B0F5A02F0DD1E0480838006840F468
:103A40008020DE49083908600846006840F480306C
:103A500008600CE0D9480838006820F48030D74965
:103A6000083908600846006820F48020086000BF1C
:103A7000606890B1FFF784FD054606E0FFF780FD22
:103A8000401B642801D903209EE7CC480838006811
:103A9000C0F340400028F1D011E0FFF771FD05466A
:103AA00006E0FFF76DFD401B642801D903208BE77A
:103AB000C24808380068C0F340400028F1D120789F
:103AC00000F0020002285FD1BC48006800F00C0042
:103AD00058B1BA48006800F00C0008281CD1B7485B
:103AE000001F006800F48000B0B9B44808380068CE
:103AF000C0F3400020B1E068012801D0012063E755
:103B0000AE480838006820F0F800216940EAC1009A
:103B1000AA490839086037E0E06800B30120A849E5
:103B20000860FFF72DFD054606E0FFF729FD401B65
:103B3000022801D9032047E7A04808380068C0F3ED
:103B400040000028F1D09D480838006820F0F800B7
:103B5000216940EAC10099490839086014E0002051
:103B600097490860FFF70CFD054606E0FFF708FDE2
:103B7000401B022801D9032026E790480838006836
:103B8000C0F340000028F1D1207800F00800082898
:103B90002CD16069A8B101208A490860FFF7F0FCC8
:103BA000054606E0FFF7ECFC401B022801D9032084
:103BB0000AE782486C300068C0F340000028F1D06A
:103BC00014E000207F490860FFF7DAFC054606E0B4
:103BD000FFF7D6FC401B022801D90320F4E6774802
:103BE0006C300068C0F340000028F1D1207800F06C
:103BF0000400042870D1002770483830006800F0B5
:103C0000805090B900BF002000906C4838300068A8
:103C100040F080506949383108600846006800F07B
:103C20008050009000BF00BF01276748006800F483
:103C30008070B0B96448006840F4807062490860E0
:103C4000FFF79EFC054606E0FFF79AFC401B0228A2
:103C500001D90320B8E65C48006800F480700028B1
:103C6000F2D000BFA068012808D15448683000682D
:103C700040F001005149683108601DE0A068052846
:103C80000DD14E486830006840F004004B4968315F
:103C900008600846006840F0010008600CE04748F2
:103CA0006830006820F00100444968310860084627
:103CB000006820F00400086000BFA068A8B1FFF70A
:103CC0005FFC054609E0FFF75BFC401B41F28831D1
:103CD000884202D9032077E626E038486830006839
:103CE000C0F340000028EED013E0FFF749FC054682
:103CF00008E0FFF745FC401B41F28831884201D9BA
:103D0000032061E62D4868300068C0F340000028B9
:103D1000EFD1012F07D129483830006820F08050BA
:103D200026493831086000BFA069002845D02348E3
:103D3000006800F00C0008285DD0A069022845D179
:103D400000201F490866FFF71BFC054606E0FFF749
:103D500017FC401B022801D9032035E61748083814
:103D60000068C0F340600028F1D1D4E9070108439E
:103D7000616A40EA81110122A06AC2EB500041EA67
:103D800000412C20005D41EA00600C49091F0860D9
:103D900001200B490866FFF7F3FB054606E0FFF735
:103DA000EFFB401B022801D903200DE60348083829
:103DB0000068C0F340600028F1D049E008380240B4
:103DC00000004742800E4742007000400020214919
:103DD0000866FFF7D5FB054606E0FFF7D1FB401B61
:103DE000022801D90320EFE51B480068C0F34060BA
:103DF0000028F2D12CE0A069012800D1E4E51648A2
:103E0000001D0668A069012820D006F48001E06941
:103E100081421BD106F03F01206A814216D147F64C
:103E2000C0703040616AB0EB811F0FD106F44031A1
:103E30000122A06AC2EB5000B1EB004F06D106F0A0
:103E400070612C20005DB1EB006F01D00120BBE55B
:103E50000020B9E5000047420038024010B5044692
:103E60000CB9012010BD606A38B96068B0F5827F76
:103E700000D105E00021E16102E0002121616161E2
:103E80000021A16294F8510028B9002084F8500064
:103E9000204600F047F8022084F8510020680068AE
:103EA00020F0400021680860A08800F48270218919
:103EB00001F404410843A18901F400610843217C15
:103EC00001F002010843217D01F001010843218B2B
:103ED00001F400710843217F01F0380108432021DB
:103EE000095D01F080010843218D01F40051084370
:103EF000216808600421A06901EA104094F82410A8
:103F000001F010010843216848602068C06920F46E
:103F100000602168C86100206065012084F85100BC
:103F200000209FE710B586B00446142101A8FCF7D5
:103F3000A9FC37492068884230D100BF002000909A
:103F40003448006840F480503249086008460068F0
:103F500000F48050009000BF00BF00BF0020009020
:103F60002C481438006840F001002A4914390860D0
:103F70000846006800F00100009000BF00BFE0208C
:103F8000019002200290002003900320049005205D
:103F9000059001A92048FFF7F3F936E01F49206892
:103FA000884232D100BF002000901A48001F0068EC
:103FB00040F480401749091F08600846006800F473
:103FC0008040009000BF00BF00BF0020009011485B
:103FD0001438006840F002000E49143908600846A1
:103FE000006800F00200009000BF00BF4FF4604086
:103FF00001900220029000200390032004900520ED
:10400000059001A90648FFF7BBF906B010BD0000F6
:1040100000300140443802400000024000380040B7
:104020000004024070B504462546681EB0F1807F4A
:1040300001D301200FE0681E4FF0E02148610F21FD
:104040004FF0FF3001F048FB00204FF0E021886185
:1040500007200861002070BDF8B504460E461746DB
:1040600094F83E00202836D106B10FB90120F8BDE2
:1040700000BF94F83C00012801D10220F7E701209D
:1040800084F83C0000BF20633A463146204601F0E8
:1040900059FA0546EDB9206B012819D100BF00205F
:1040A000009020680068009020684068009000BF81
:1040B00000BF00BF00BF21680C3151E8001F41F074
:1040C000100021680C3141E80002002AF3D100E021
:1040D00001252846CBE70220C9E7000070B5044659
:1040E0000D460C492068884203D10B4801F045FD7C
:1040F0000EE00A492068884203D1094801F03DFDDD
:1041000006E008492068884202D1074801F035FDE1
:1041100070BD000000100140680100200044004014
:10412000B8010020004C00400802002070B5044691
:10413000002520684069C0F3C01594F83D0021288F
:1041400017D1B5B100BF00BF2168143151E8001F7D
:1041500021F080002168143141E80002002AF3D1E7
:1041600000BF606B10B1606BFEF7E6FD204601F00A
:1041700044F820684069C0F3801594F83E00222876
:1041800017D1B5B100BF00BF2168143151E8001F3D
:1041900021F040002168143141E80002002AF3D1E7
:1041A00000BFA06B10B1A06BFEF7C6FD204600F06B
:1041B000DEFF002070BD000038B5044600252B4905
:1041C0002068884201D12A4D0AE02A4920688842A5
:1041D00001D1294D04E029492068884200D1284DA9
:1041E000206C00F0020050B100BF00200090206859
:1041F0000068009020684068009000BF00BF206CFD
:1042000000F0040050B100BF00200090206800685A
:10421000009020684068009000BF00BF20680068E0
:10422000C0F3C00050B100BF0020009020680068BB
:10423000009020684068009000BF00BF20680068C0
:10424000C0F3400050B100BF00200090206800681B
:10425000009020684068009000BF00BF25B1EA8B45
:10426000A9696868FFF7F8FE38BD0000001001403A
:104270006801002000440040B8010020004C0040CC
:10428000080200202DE9F84F0446206805682068E0
:10429000C668206847694FF00009CA4605F00F0953
:1042A000B9F1000F0AD105F0200038B106F0200066
:1042B00020B1204600F0B4FFBDE8F88FB9F1000F3F
:1042C0007CD007F0010018B906F49070002875D072
:1042D00005F0010030B106F4807018B1206C40F098
:1042E0000100206405F0040030B107F0010018B1AE
:1042F000206C40F00200206405F0020030B107F0AD
:10430000010018B1206C40F00400206405F00800A2
:1043100048B106F0200010B907F0010018B1206C78
:1043200040F008002064206C002846D005F02000F2
:1043300028B106F0200010B1204600F071FF20687F
:104340004069C0F3801A206C00F0080010B9BAF17F
:10435000000F2DD0204600F00AFF2068406900F0D1
:104360004000402820D100BF00BF2168143151E82F
:10437000001F21F040002168143141E80002002AAA
:10438000F3D100BFA06B50B17548A16B0865A06B5D
:10439000FEF728FD88B1A06B016D88470DE020462F
:1043A000FFF70AFF09E009E02046FFF705FF04E0F8
:1043B0002046FFF701FF002020647DE7206B0128E5
:1043C00076D105F01000002872D006F01000002809
:1043D000FAD000BF0020009020680068009020689C
:1043E0004068009000BF00BF2068406900F04000B6
:1043F00040285ED1A06B006840681FFA80F8B8F1D1
:10440000000F54D0A08D404551DDA4F82E80A06B44
:10441000C069B0F5807F43D000BF00BF21680C3178
:1044200051E8001F21F4807021680C3141E800023E
:10443000002AF3D100BF00BF00BF2168143151E84A
:10444000001F21F001002168143141E80002002A18
:10445000F3D100BF00BF00BF2168143151E8001F35
:1044600021F040002168143141E80002002AF3D114
:1044700000BF202084F83E000020206300BF00BF62
:1044800021680C3151E8001F21F0100021680C3127
:1044900041E80002002AF3D100BFA06BFEF74CFCFC
:1044A000A08DE28D801A81B22046FFF717FE03E748
:1044B00040E0A08DE18D401A1FFA80F8E08DC0B376
:1044C000B8F1000F35D000BF00BF21680C3151E8B2
:1044D000001F21F4907021680C3141E80002002A8D
:1044E000F3D100BF00BF00BF2168143151E8001FA5
:1044F00021F001002168143141E80002002AF3D1C3
:1045000000BF202084F83E000020206300BF00BFD1
:1045100021680C3151E8001F21F0100021680C3196
:1045200041E80002002AF3D100BF41462046FFF7D0
:10453000D5FDC1E605F0800030B106F0800018B16D
:10454000204601F067F8B7E605F0400030B106F00C
:10455000400018B1204600F040FEADE600BFABE6DB
:10456000D54F000810B504460CB9012010BDA06954
:1045700000B100E000BF94F83D0028B9002084F8A5
:104580003C00204600F028F8242084F83D002068F4
:10459000C06820F400502168C860204600F0BCFECE
:1045A0002068006920F49040216808612068406913
:1045B00020F02A00216848612068C06840F400505B
:1045C0002168C86000202064202084F83D0084F821
:1045D0003E000020CAE7000010B586B00446142152
:1045E00001A8FCF74FF9F849206888427AD100BF4A
:1045F00000200090F548006840F40020F34908606E
:104600000846006800F40020009000BF00BF00BF13
:1046100000200090ED481038006840F00100EB49A0
:10462000103908600846006800F00100009000BFE3
:1046300000BF03200190022002900020039003207D
:1046400004900820059001A9E148FEF799FEE14891
:10465000E1490860400548600021DF488160C16091
:104660004FF480610161002141618161C1614FF4BA
:104670004031016200214162FEF7E8FC08B1FEF71B
:10468000FFF900BFD448A063846300BFD148303035
:10469000D24908604FF0006048604021CF488160F7
:1046A0000021C1604FF4806101610021416181619D
:1046B000C1614FF40031016200214162FEF7C6FC86
:1046C00008B1FEF7DDF900BFC4486063846300BF32
:1046D000002201213420FEF7E1FF3420FEF7CEFF57
:1046E0006FE1FFE7BE49206888427DD100BF00200E
:1046F0000090B648001D006840F01000B349091D45
:1047000008600846006800F01000009000BF00BF7D
:1047100000BF00200090AD481038006840F0020053
:10472000AA49103908600846006800F002000090AD
:1047300000BF00BFC0200190022002900020039023
:10474000032004900720059001A9A648FEF718FE53
:10475000A548A64908604FF0006048600021A348C2
:104760008160C1604FF4806101610021416181611C
:10477000C1614FF48031016200214162FEF766FCA5
:1047800008B1FEF77DF900BF9848A063846300BFBD
:1047900095487830964908604FF0006048604021A5
:1047A000934881600021C1604FF480610161002164
:1047B00041618161C1614FF4803101620021416238
:1047C000FEF744FC08B1FEF75BF900BF8848606360
:1047D000846300BF002201212520FEF75FFF252012
:1047E000FEF74CFFEDE0FFE78249206888427CD16C
:1047F00000BF002000907548006840F40030734905
:1048000008600846006800F40030009000BF00BF58
:1048100000BF002000906D481038006840F0010093
:104820006A49103908600846006800F001000090ED
:1048300000BF00BF0C2001900220029000200390D6
:10484000032004900720059001A96148FEF798FD18
:1048500060484830684908604FF0006048600021B7
:1048600065488160C1604FF4806101610021416150
:104870008161C1614FF44031016200214162FEF764
:10488000E5FB08B1FEF7FCF800BF5B48A06384635A
:1048900000BF50486030594908604FF000604860E0
:1048A0004021564881600021C1604FF48061016160
:1048B000002141618161C1614FF400310162002139
:1048C0004162FEF7C3FB08B1FEF7DAF800BF4B48C0
:1048D0006063846300BF002201212620FEF7DEFE14
:1048E0002620FEF7CBFE6CE0FFE7454920688842B2
:1048F00031D100BF002000903448006840F480208F
:10490000324908600846006800F48020009000BF2B
:1049100000BF00BF002000902C481038006840F015
:1049200002002A49103908600846006800F00200B9
:10493000009000BF00BF4FF4406001900220029041
:1049400000200390032004900720059001A925482A
:10495000FEF716FD35E02B492068884231D100BFB3
:10496000002000901948001D006840F02000174901
:10497000091D08600846006800F02000009000BF94
:1049800000BF00BF0020009010481038006840F0C1
:1049900004000E49103908600846006800F0040061
:1049A000009000BF00BFC0200190022002900020B4
:1049B0000390032004900820059001A91248FEF7F7
:1049C000DFFC06B010BD0000004C00404038024043
:1049D00000000240406002409C040020FC040020D3
:1049E0000010014000040240406402405C050020C9
:1049F000BC050020004400401C0600207C0600206E
:104A00000048004000140140000802407047704711
:104A1000F7B50446154694F83D00202846D1019884
:104A200000B10DB90120FEBD00BF94F83C00012883
:104A300001D10220F7E7012084F83C0000BF019873
:104A40002062A584E58400202064212084F83D00B4
:104A50001748616BC8631748616B08641648616B3F
:104A6000C8640020616B086501AE23681A1D3168B7
:104A70002B46606BFEF760FB6FF04000216808601A
:104A800000BF002084F83C0000BF00BF00BF2168C9
:104A9000143151E8001F41F080002168143141E8D1
:104AA0000002002AF3D100BF0020BCE70220BAE7D1
:104AB0000951000861510008E94F000810B504468B
:104AC0000B492068884203D10A4801F0F1F80EE052
:104AD00009492068884203D1084801F0E9F806E056
:104AE00007492068884202D1044801F0E1F810BD6E
:104AF000001001406801002000440040B80100207F
:104B0000004C0040704700BFFEE7000008B500BF42
:104B1000002000902648006840F4001024490860F6
:104B20000846006800F40010009000BF00BF00BFFE
:104B3000002000900846006840F4800008600846A5
:104B4000006800F48000009000BF00BF0022114602
:104B50000D20FEF7A3FD0D20FEF790FD002211466B
:104B60000F20FEF79BFD0F20FEF788FD0022114667
:104B70001020FEF793FD1020FEF780FD0022114665
:104B80001120FEF78BFD1120FEF778FD0022114663
:104B90003A20FEF783FD3A20FEF770FD0022114611
:104BA0004620FEF77BFD4620FEF768FD08BD0000AD
:104BB0003038024000B587B0142102A8FBF762FE2E
:104BC00000BF002001904F48006840F080004D4930
:104BD00008600846006800F08000019000BF00BF38
:104BE00000BF002001900846006840F00100086006
:104BF0000846006800F00100019000BF00BF00BF40
:104C0000002001900846006840F004000860084653
:104C1000006800F00400019000BF00BF00BF00204A
:104C200001900846006840F01000086008460068DF
:104C300000F01000019000BF00BF00BF00200190F5
:104C40000846006840F0020008600846006800F06E
:104C50000200019000BF00BF00BF00200190084685
:104C6000006840F0080008600846006800F008008E
:104C7000019000BF00BF002230212348FEF77AFCDC
:104C800000224FF400612148FEF774FC00224FF42B
:104C900088511F48FEF76EFC002238211D48FEF7A0
:104CA00069FC3020029001200390002004900590C0
:104CB00002A91548FEF764FB4FF400600290012042
:104CC000039000200490059002A91048FEF758FBBD
:104CD0004FF488500290012003900020049005902A
:104CE00002A90B48FEF74CFB3820029001200390EC
:104CF00000200490059002A90648FEF741FB07B08A
:104D000000BD0000303802400008024000100240A0
:104D100000040240000C024010B50E480E49086025
:104D20004FF48270486000210B488160C1600161CE
:104D300041614FF4007181610021C16101624162F2
:104D400081620A21C162FFF789F808B1FDF798FE78
:104D500010BD0000003001409802002010B50E4840
:104D60000E4908604FF48270486000210B48816052
:104D7000C160016141614FF4007181610021C16135
:104D80000162416281620A21C162FFF767F808B1DE
:104D9000FDF776FE10BD000000380040F002002054
:104DA00010B50B480B4908604FF4E1304860002112
:104DB00008488160C16001610C214161002181616D
:104DC000C161FFF7CFFB08B1FDF75AFE10BD00002F
:104DD000004C00404803002010B50B480B49086008
:104DE0004FF4E1304860002108488160C1600161F2
:104DF0000C21416100218161C161FFF7B3FB08B162
:104E0000FDF73EFE10BD0000001001408C030020A5
:104E100010B50B480B4908604FF4E13048600021A1
:104E200008488160C16001610C21416100218161FC
:104E3000C161FFF797FB08B1FDF722FE10BD00002E
:104E400000440040D003002010B50B480B49086017
:104E50004FF4E1304860002108488160C160016181
:104E60000C21416100218161C161FFF77BFB08B129
:104E7000FDF706FE10BD00000048004014040020AD
:104E800010B50B480B4908604FF4E1304860002131
:104E900008488160C16001610C214161002181618C
:104EA000C161FFF75FFB08B1FDF7EAFD10BD00002F
:104EB000001401405804002000BFFEE700BFFEE7D9
:104EC0007047704710B50948416901208847084874
:104ED0000121426C904707480121426C90470648E7
:104EE0000121426C9047FEF751FB10BD8C00002061
:104EF00068010020B80100200802002000B593B02E
:104F0000302107A8FBF7BEFC142102A8FBF7BAFC6E
:104F100000BF002001902448006840F080502249E2
:104F200008600846006800F08050019000BF00BF94
:104F300000BF002001901D48006840F480401B49DC
:104F400008600846006800F48040019000BF00BF80
:104F5000012007900004089002200D9041050E9159
:104F600004210F91A8211091022111910421129185
:104F700007A8FEF725FD08B1FDF782FD0F2002907E
:104F800002200390002004904FF4A05005904FF4AD
:104F900080500690052102A8FEF7D2FB08B1FDF76C
:104FA0006FFD13B000BD00004038024000700040AB
:104FB0000348006840F47000014908607047000031
:104FC00088ED00E010B50248FFF75CF910BD000065
:104FD0004803002070B50546AC6B0020E085E084F6
:104FE0002046FFF7E9F870BD70B506460025B46BA2
:104FF00020684069C0F3C01594F83D00212805D110
:1050000025B10020E084204600F0F7F820684069D0
:10501000C0F3801594F83E00222805D125B1002068
:10502000E085204600F0A3F8206C40F010002064DA
:105030002046FFF7C1F870BD70B50546AC6B286817
:10504000006800F48070002842D1E08500BF00BFF6
:1050500021680C3151E8001F21F4807021680C3167
:1050600041E80002002AF3D100BF00BF00BF216861
:10507000143151E8001F21F001002168143141E88A
:105080000002002AF3D100BF00BF00BF2168143125
:1050900051E8001F21F040002168143141E800026E
:1050A000002AF3D100BF202084F83E00206B0128A5
:1050B0000ED100BF00BF21680C3151E8001F21F064
:1050C000100021680C3141E80002002AF3D100BF32
:1050D000206B012804D1A18D2046FEF7FFFF02E0DE
:1050E0002046FFF793FC70BD70B50546AC6B206B96
:1050F000012805D1A08D41082046FEF7EFFF02E010
:105100002046FFF784FC70BD70B50546AC6B28687F
:10511000006800F48070F8B90020E08400BF00BF90
:105120002168143151E8001F21F0800021681431FA
:1051300041E80002002AF3D100BF00BF00BF216890
:105140000C3151E8001F41F0400021680C3141E86A
:105150000002002AF3D102E02046FFF7AFFC70BD49
:1051600070B50446A56B2846FFF7CCFC70BD00BFA8
:1051700000BF02680C3252E8002F22F490710268DE
:105180000C3242E80013002BF3D100BF00BF00BF78
:105190000268143252E8002F22F001010268143232
:1051A00042E80013002BF3D100BF016B01290ED19F
:1051B00000BF00BF02680C3252E8002F22F010013D
:1051C00002680C3242E80013002BF3D100BF20210B
:1051D00080F83E1000210163704710B50446206836
:1051E000C06820F040002168C860202084F83D009D
:1051F0002046FFF763FC002010BD00BF00BF02681F
:105200000C3252E8002F22F0C00102680C3242E852
:105210000013002BF3D100BF202180F83D10704710
:10522000F8B5044694F83E00222873D1A068B0F582
:10523000805F0CD1206950B90025A66A20684068BB
:10524000C0F308003080A06A801CA06215E0A56A47
:105250000026A068B0F5805F03D0A06828B9206957
:1052600018B920684068287004E02068406800F0A1
:105270007F002870A06A401CA062E08D401E80B2B2
:10528000E085002844D12068C06820F02000216813
:10529000C8602068C06820F480702168C8602068F9
:1052A000406920F0010021684861202084F83E0018
:1052B000206B012826D10020206300BF00BF216899
:1052C0000C3151E8001F21F0100021680C3141E839
:1052D0000002002AF3D100BF2068006800F010002F
:1052E00010280AD100BF00200090206800680090BC
:1052F00020684068009000BF00BFA18D2046FEF7E7
:10530000EDFE02E02046FFF781FB0020F8BD01E042
:105310000020FBE70220F9E72DE9F84F044620685A
:10532000006920F44050E168084321680861216960
:10533000A068084361690843E16908430090206858
:10534000C06849F20C618843009908432168C8602D
:105350002068406920F44070A169084321684861D1
:1053600076492068884203D075492068884203D175
:10537000FEF7BEFA814602E0FEF7AAFA8146E0692E
:10538000B0F5004F6CD102206168A0FB01500346CC
:105390001920A9FB007001462A463846FAF7E2FFB9
:1053A0006421B0FBF1F04FEA001A02206168A0FB13
:1053B00001510B461920A9FB00712A463846FAF71D
:1053C000D1FF834602206168A0FB015003461920EB
:1053D000A9FB00712A463846FAF7C4FF6421B0FBE6
:1053E000F1F000EBC00101EB0010ABEB80003221CB
:1053F00001EBC0006421B0FBF1F000F0F8000AEB13
:10540000400A02206168A0FB015003461920A9FB55
:10541000007001462A463846FAF7A4FF8346022068
:105420006168A0FB015003461920A9FB00712A46C0
:105430003846FAF797FF6421B0FBF1F000EBC001AA
:1054400001EB0010ABEB8000322101EBC0006421C6
:10545000B0FBF1F000F007005044216888606AE07A
:1054600004206168A0FB015003461920A9FB0070CD
:1054700001462A463846FAF775FF824604206168DD
:10548000A0FB015003461920A9FB007001462A46E3
:105490003846FAF767FF6421B0FBF1F000EBC0017A
:1054A00001EB0010AAEB8000322101EB0010642117
:1054B000B0FBF1F000F0F00A04206168A0FB01707D
:1054C00003461920A9FB00513A462846FAF74AFF3D
:1054D0006421B0FBF1F00AEB001A04206168A0FB24
:1054E00001510B461920A9FB00712A463846FAF7EC
:1054F00039FF834604206168A0FB01500346192050
:10550000A9FB007001462A463846FAF72BFF6421B2
:10551000B0FBF1F000EBC00101EB0010ABEB800041
:10552000322101EB00106421B0FBF1F000F00F001C
:10553000504421688860BDE8F88F000000100140E9
:105540000014014077B581B0044615460298A06268
:10555000A58500202064222084F83E002A48A16B03
:10556000C8632A48A16B08642948A16BC86400205D
:10557000A16B086502AE32682368191D2B46A06B2B
:10558000FDF7DAFD00BF0020009020680068009061
:1055900020684068009000BF00BF00BF002084F872
:1055A0003C0000BF206970B100BF00BF21680C3112
:1055B00051E8001F41F4807021680C3141E800027D
:1055C000002AF3D100BF00BF00BF2168143151E8A9
:1055D000001F41F001002168143141E80002002A57
:1055E000F3D100BF00BF00BF2168143151E8001F94
:1055F00041F040002168143141E80002002AF3D153
:1056000000BF002004B070BD39500008E950000808
:10561000E94F0008014691F83D00212828D188680B
:10562000B0F5805F0BD1086948B90A6A1088C0F3E9
:1056300008000B685860086A801C086205E00B6A65
:10564000581C086218780B685860C88C401E80B2DD
:10565000C88458B90868C06820F080000B68D8601A
:105660000868C06840F040000B68D86000207047B0
:105670000220FCE710B50248FEF704FE10BD000052
:105680008C03002010B50248FEF7FCFD10BD0000A1
:10569000D003002000BFFEE703B40198410000984A
:1056A00050EAC12018BF04204A0D18BF40F0010085
:1056B00040F2FF72B2EB515F08BF40F002000128D8
:1056C00008BF052002B0704702480068C0F30220FE
:1056D000704700000CED00E010B5002804DB0A075D
:1056E000130E054A135406E00A07140E034A00F08D
:1056F0000F031B1FD45410BD00E400E018ED00E0C0
:1057000030380A2801D2012070470020704700007D
:1057100010B50D49086A80470C48416B88470C4812
:10572000416B88470B48416B88470B4908688047A5
:105730000A480B49C268082090470A4948688047D0
:1057400009490868804710BDEC000020680100206E
:10575000B801002008020020E00000208C0000209A
:105760002C00002080020020A800002010B5034972
:105770000869804701F0ECFA10BD00008C000020A1
:10578000034A12689080024A1268916070470000D4
:10579000A400002010B51A480068806800B910BD48
:1057A000002425E016480068806804EB440110F8E6
:1057B0002100D0B1002012490968896804EB440235
:1057C00001F822000E480068806804EB440100EBF9
:1057D0008100806800B909E009490968896804EB1B
:1057E000440201EB82018868804700BF601C84B2DC
:1057F000034800688088A042D4DC00BFCFE70000E7
:10580000A400002010B501462F4A12681288521CCD
:105810002D4B1B681A802C4A12681288B2F57A7FC9
:1058200006DB294A12685288521C274B1B685A8093
:10583000254A1268926802B910BD00203CE0224A55
:105840001268926800EB400302EB830252888AB32D
:105850001D4A1268926800EB400302EB83025288F3
:10586000521E194B1B689B6800EB400403EB84033A
:105870005A80154A1268926800EB400302EB8302DB
:105880005288BAB90122104B1B689B6800EB400498
:1058900003F824200C4A1268926800EB400302EBE4
:1058A00083029288084B1B689B6800EB400403EB63
:1058B00084035A80421C90B2034A12689288824242
:1058C000BDDC00BFB8E70000A4000020014800785C
:1058D00070470000DC00002010B50020024908706D
:1058E00000F004F810BD0000DC00002030B50446D4
:1058F0000021102900DB30BD094D2970094D6A5C7B
:10590000094D6B5C002001E0451CE8B20428FBDB7C
:10591000002001E0451CE8B21028FBDB00BFEAE7ED
:10592000DC000020BC000020CC00002010B586B0B8
:105930000446002001900B200390012004900220D7
:10594000059000200090694601A8FDF753FC06B0C1
:1059500010BD000010B5064948688047102205496F
:10596000054800F055F802494868804710BD00001E
:10597000B0000020FC00002000000E0870B51022CE
:105980000E49A1F11000FAF7CBFEA8B10C49486806
:10599000804772B6102209490A4800F05DF80446B3
:1059A0002CB906481038054610352ECD2EC062B6EB
:1059B00003494868804700BF70BD0000FC0000201C
:1059C000B000002000000E0810B5FFF7D7FF10BD93
:1059D00010B5FFF7BFFF0C480068808BB0F57A7FE9
:1059E00003DD282108480068818307480068C08BD0
:1059F000102803DD102104480068C18303480446D1
:105A000010341ECC1EC010BD1C010020EC00002074
:105A10002DE9F84103460C4621461D46960802F042
:105A20000307002005E055F820C0C1F800C0091D9B
:105A3000401CB042F7D36FB155F826000090EC46F9
:105A4000002004E01CF8008001F80080401CB842EF
:105A5000F8D300BFBDE8F8812DE9FC5F0746884612
:105A6000154600244646A808019005F00309BA46E9
:105A7000FDF76CFC3846FFF759FF044624B1FDF7EB
:105A80000FFC2046BDE8FC9F4FF0000B0FE0D6F85E
:105A900000C06246002351460220FDF70BFC04467D
:105AA00004B107E00AF1040A361D0BF1010B01985D
:105AB0008345ECD300BFB4B9B9F1000F13D04FF058
:105AC000FF300090EB46002003E0315C0BF8001043
:105AD000401C4845F9D3002351460220009AFDF7A7
:105AE000E9FB044600BFFDF7DBFB2046CAE7704731
:105AF000704710B5002404E0322000F0DCF8601C90
:105B0000C4B2142CF8DB10BD70472DE9F0410446F7
:105B1000884617460020A074A08BB84200DAA78BF5
:105B20003A4641466069FAF746FE3A46616960685E
:105B3000FEF76EFFFDF724FD054608E0FDF720FDAA
:105B40000646701BC82802D90120A07402E0A07C80
:105B50000028F3D000BFBDE8F08110B504466068AE
:105B60000068C06840F0100061680968C860E28B96
:105B7000A1696068FEF770FA10BD70B504466068F0
:105B8000FEF7D4FAE08BE16809684968401A86B2EA
:105B900006B970BD002506E0A2695119206801F020
:105BA0009CF8681C85B2B542F6DB204600F042F84E
:105BB000E28BA1696068FEF74FFA00BFE9E70000D9
:105BC00070B50446A08C618C884227DA20688089F1
:105BD0002084204600F034F8208CE18B88421DDCC4
:105BE000208CD8B1208C40F6B831884203D9206887
:105BF00001F027F812E0002506E0094A5119206853
:105C000001F027F8681C85B2208CA842F5DCA06C56
:105C100020B1218C22460248A36C984770BD000039
:105C2000407B002090F82620012A02D1428C0A44B1
:105C300042847047012180F826100021418470477A
:105C4000002180F826104184704700002DE9F041C2
:105C500004460F4616461448844204D1012211021C
:105C60001248FDF787FCA08B96FBF0F01FFA80F836
:105C7000002507E0A28B02FB05712046FFF745FFD8
:105C8000681C85B24545F5DBA08B00FB156086B22C
:105C90000EB9BDE8F081A08B00FB057132462046AD
:105CA000FFF733FF00BFF4E70802002000040240C2
:105CB00001218174704710B504462046FDF786FA2D
:105CC00010BD8A68002A01DCFBF730BE521E8A60D4
:105CD0004A68C0B2531C4B60107070472DE9F84FF2
:105CE00004460D469046052D01DABDE8F88F207870
:105CF000AA2802D16078552800D0F6E7681E215CFA
:105D0000A81E205C41EA002BA81E81B2204600F0AC
:105D10007AFF0746381240EA072087B25F4500D075
:105D2000E3E7A678032E01D1102E00D0DDE794F82A
:105D3000039094F804A0601D00901B48C0F80080F8
:105D4000A9F1100008282BD2DFE800F0040A101691
:105D5000171D232951463046009A00F027FD1FE009
:105D600051463046009A00F021F819E0514630467D
:105D7000009A00F0E5FA13E012E051463046009A2E
:105D800000F0DAFC0CE051463046009A00F08EFE3E
:105D900006E051463046009A00F09CFC00E000BF4F
:105DA00000BF00BFA1E700007C0200202DE9F74FF3
:105DB00090B000254FF40061FE48FAF741FDAB4674
:105DC00000200F902AE00F9800EB8001FA4810F8AD
:105DD0003100012800D01DE0002617E00F9901EBEB
:105DE0008102F54901EBC201183131F826004FF26A
:105DF0000301014041B105AA0F9902F80B100BF104
:105E0000010101F0FF0B03E0701C86B2042EE5DBFC
:105E100000BF00BF0F98401C80B20F900F98202841
:105E2000D1DB58464FEAEB710BEB9171C1F387015F
:105E30000E914FEAEB710BEB91718910ABEB810185
:105E4000C9B20D910D99002903DD0E98401CC0B216
:105E50000E901098032877D11198012802D00328BA
:105E600073D108E2D548006881780E98401E8142BF
:105E70006CD10D98002869DD4FF00008E7E0CF48AD
:105E80000068807808EB80001FFA80FA05A810F8F7
:105E90000A90444600270AEB8A01C74800EBC1007C
:105EA0000D30C44B5A19791C631C009098B2C4A3DE
:105EB00000F02EFE054601270AEB8A01BE4800EBE2
:105EC000C1008078BB4B5A19791C631C009098B2B2
:105ED000BBA300F01DFE054602270AEB8A01B64867
:105EE00000EBC100C01CB34B5A19791C631C009015
:105EF00098B2B3A300F00CFE0546032700200490DF
:105F000000260FE009EB8901AB4800EBC100183017
:105F100030F8260000F4704010B10020049003E037
:105F2000701C86B2042EEDDB00BF049800F47040B4
:105F300068B1A04B5A197B1C99B2631C98B2A1A3FB
:105F400000F0E6FD05460CE0CCE1BEE184E0994BB3
:105F50005A197B1C99B2631C98B29CA300F0D8FD1F
:105F6000054600266DE009EB8901934800EBC1006E
:105F7000183030F82600039009EB89018E4800EBB9
:105F8000C100183000EB86004088029006EB460006
:105F9000001D87B2039800F0010050B1854B5A19DB
:105FA0007B1C99B2631C98B28AA300F0B1FD054630
:105FB00009E0804B5A197B1C99B2631C98B283A3E9
:105FC00000F0A6FD054606EB4600401D87B203988B
:105FD00000F0020050B1774B5A197B1C99B2631C38
:105FE00098B27EA300F094FD054609E0714B5A1962
:105FF0007B1C99B2631C98B274A300F089FD05461E
:1060000006EB4600801D87B2039800F0010060B1E6
:106010000298684B5A197B1C99B2631C009098B285
:1060200070A300F075FD054609E0624B5A197B1C10
:1060300099B2631C98B26CA300F06AFD0546701C0F
:1060400086B2042E8FDB08F101001FFA80F80D984C
:106050008045FFF614AF0DE14FF0000806E1574808
:106060000068807808EB80001FFA80FA05A810F815
:106070000A904446002709EB89014F4800EBC10014
:106080000D304C4B5A19791C631C009098B24CA3EC
:1060900000F03EFD054601270AEB8A01464800EB69
:1060A000C1008078434B5A19791C631C009098B248
:1060B00043A300F02DFD054602270AEB8A013E4866
:1060C00000EBC100C01C3B4B5A19791C631C0090AB
:1060D00098B23BA300F01CFD054603270020049066
:1060E00000260FE009EB8901334800EBC1001830AE
:1060F00030F8260000F4704010B10020049003E056
:10610000701C86B2042EEDDB00BF049800F47040D2
:1061100050B1284B5A197B1C99B2631C98B229A321
:1061200000F0F6FC054609E0224B5A197B1C99B297
:10613000631C98B225A300F0EBFC054600268EE018
:1061400009EB89011C4800EBC100183030F826002B
:10615000039009EB8901184800EBC100183000EBEF
:1061600086004088029006EB4600001D87B2039827
:1061700000F0010050B10F4B5A197B1C99B2631CFF
:1061800098B214A300F0C4FC054609E0094B5A1963
:106190007B1C99B2631C98B20CA300F0B9FC0546B5
:1061A00006EB4600401D87B2039800F0020040B3A2
:1061B000004B1BE0F8860020BE0C00208802002067
:1061C00025730000B3ACCAB100000000D5FDB3A335
:1061D00000000000C2A9D2BA00000000B6CFB4F897
:1061E0000000000025640000300000005A197B1CEC
:1061F00099B2631C98B2AFF21C0300F089FC05460B
:106200000AE0444B5A197B1C99B2631C98B2AFF256
:10621000440300F07DFC054606EB4600801D87B276
:10622000039800F0010068B102983A4B5A197B1CA0
:1062300099B2631C009098B2AFF2580300F068FC6A
:1062400005460AE0334B5A197B1C99B2631C98B27D
:10625000AFF26C0300F05CFC0546701C86B2042EA5
:10626000FFF66EAF08F101001FFA80F8B8F1040FD5
:10627000FFF6F5AE2CE012980078012813D10E98A5
:10628000401E254909688978884204DC002022499B
:106290000968887018E0204800688078401C1E4912
:1062A0000968887010E01C480068807828B90E984A
:1062B000401E19490968887006E017480068807810
:1062C000401E15490968887000BF13B0BDE8F08F03
:1062D00000BF1048FAF750FA85B229460D4800F081
:1062E0001DF814E01098102811D11198012802D03F
:1062F000022802D100E001E000E0E6E700BF054827
:10630000FAF73AFA85B22946024800F007F800BFCA
:10631000DBE70000F88600208802002070B5044604
:106320000D460648006838B1044800682A462146F0
:10633000836B02480068984770BD00007C02002013
:106340002DE9F74F8AB000244FF40061D248FAF7E4
:1063500077FA9BF80300C11700EB9171891008913F
:106360009BF80300C11700EB91718910A0EB81012C
:10637000C9B207910798002803DD0898401CC0B2F5
:1063800008900A9803287DD10B98012802D0032891
:1063900079D130E10C98007805900598012802DB4E
:1063A0000598042801DD012005900598401EBB4991
:1063B0000968097800EB810000F0FF08B848007810
:1063C000404501DC4FF00008B44800684078404583
:1063D00003D00020B1490968C870B048006880F84F
:1063E0000180C8EBC80000EB0811AD48801C00EB31
:1063F000410BAA480068C0788006000E0490A748A8
:106400000068C1780898401E814205D1079800288D
:1064100002DD0798069001E0042006904FF0000985
:10642000E3E00498484480B209909BF8031009986F
:10643000814200DCDDE00BF10E00099910F801A0AB
:106440004D4600270AEB8A01964800EBC100807890
:10645000914B1A19791C6B1C009098B292A300F012
:1064600057FB204484B201270AEB8A018D4800EBD8
:10647000C100C01C884B1A19791C6B1C009098B283
:106480008AA301E0FDE0F3E000F042FB204484B287
:1064900002270020039000260FE00AEB8A018148C2
:1064A00000EBC100183030F8260000F4704010B145
:1064B0000120039003E0701C86B2042EEDDB00BFC8
:1064C000039858B1744B1A197B1C99B26B1C98B283
:1064D00077A300F01DFB204484B20AE06E4B1A192A
:1064E0007B1C99B26B1C98B273A300F011FB204483
:1064F00084B2002673E00AEB8A016A4800EBC1000F
:10650000183030F8260002900AEB8A01654800EB4B
:10651000C100183000EB86004088019006EB460071
:10652000C01C87B2029800F0010058B15A4B1A19EA
:106530007B1C99B26B1C98B261A300F0E9FA20446D
:1065400084B20AE0544B1A197B1C99B26B1C98B2A6
:1065500059A300F0DDFA204484B206EB4600001D8A
:1065600087B2029800F0020058B14B4B1A197B1CFD
:1065700099B26B1C98B254A300F0CAFA204484B2BA
:106580000AE0454B1A197B1C99B26B1C98B24AA3BE
:1065900000F0BEFA204484B206EB4600401D87B2EC
:1065A000029800F0010068B101983B4B1A197B1C5E
:1065B00099B26B1C009098B23BA300F0A9FA20445A
:1065C00084B20AE0344B1A197B1C99B26B1C98B246
:1065D0003FA300F09DFA204484B2701C86B2042EC2
:1065E00089DB09F101001FFA80F906988145FFF661
:1065F00018AF00BF3DE02948006890F801802848A6
:106600000078404502DC0DB0BDE8F08FC8EBC80053
:1066100000EB08112248801C00EB410B0C9800781D
:10662000012813D10898401E1C490968C97888427E
:1066300004DC002019490968C87018E01748006890
:10664000C078401C15490968C87010E013480068FC
:10665000C07828B90898401E10490968C87006E03B
:106660000E480068C078401E0C490968C870CAE727
:10667000C9E700BF002C0DDD21460748FFF74EFE9D
:1066800008E00A98102805D10B98012800D100E0F5
:10669000B9E700BF00BFB6E7F886002088020020F7
:1066A000FC060020BE0C00202564000025730000BD
:1066B000B3ACCAB100000000D5FDB3A300000000D8
:1066C000C2A9D2BA00000000B6CFB4F800000000A2
:1066D000300000002DE9F04104460D461746002623
:1066E000032C12D1012D02D0032D02D100E002E0D3
:1066F00001E0BDE8F08100BF0E48FAF73DF886B230
:1067000031460C48FFF70AFE12E0102C10D1012D83
:1067100002D0022D02D100E001E000E0E9E700BF75
:106720000448FAF729F886B231460248FFF7F6FD29
:1067300000BFDEE7F88600202DE9F04104460D4653
:1067400017460026032C12D1012D02D0032D02D1B1
:1067500000E002E001E0BDE8F08100BF0E48FAF77A
:106760000BF886B231460C48FFF7D8FD12E0102C2A
:1067700010D1012D02D0022D02D100E001E000E095
:10678000E9E700BF0448F9F7F7FF86B2314602484F
:10679000FFF7C4FD00BFDEE7F8860020014802498C
:1067A00088647047DD5C0008680100202DE9F74F20
:1067B00082B082468B4600274FF40061B648FAF754
:1067C0003FF8B6490878C11700EB91714FEAA1096B
:1067D000B2490878C11700EB91718910A0EB8101D3
:1067E000C9B201910198002803DD09F1010000F010
:1067F000FF09BAF1030F7DD1BBF1010F03D0BBF14B
:10680000030F78D106E1A64800680178A9F10100DC
:10681000814271D1019800286EDD00247AE0A04801
:106820000068007804EB800086B225464FF000082F
:10683000C6EBC60000EB06119848801C00EB410037
:10684000001D954BDA1908F101012C466B1C0090D4
:1068500098B294A300F05CF907464FF00108C6EB2C
:10686000C60000EB06118D48801C00EB4100C0788B
:10687000894BDA1908F101016B1C009098B28AA3C8
:1068800000F046F907464FF00208C6EBC60000EBE1
:1068900006118248801C10F811007F4BDA1908F1AC
:1068A00001016B1C009098B27FA300F031F90746FC
:1068B0004FF00308C6EBC60000EB06117748801CBA
:1068C00000EB41004078744BDA1908F101016B1CB0
:1068D000009098B274A300F01BF907464FF004082B
:1068E000C6EBC60000EB06116C48801C00EB4100B3
:1068F000807802E0C5E0B7E010E0674BDA1908F1F4
:1069000001016B1C009098B267A300F001F90746E3
:10691000601C84B20198844281DB7AE0002476E036
:106920005F480068007804EB800086B225464FF08F
:106930000008C6EBC60000EB06115848801C00EBAF
:106940004100001D544BDA1908F101012C466B1C63
:10695000009098B253A300F0DBF807464FF001080F
:10696000C6EBC60000EB06114C48801C00EB410052
:10697000C078494BDA1908F101016B1C009098B2FC
:1069800049A300F0C5F807464FF00208C6EBC60061
:1069900000EB06114148801C10F811003E4BDA193B
:1069A00008F101016B1C009098B23FA300F0B0F811
:1069B00007464FF00308C6EBC60000EB0611374848
:1069C000801C00EB41004078334BDA1908F10101DB
:1069D0006B1C009098B234A300F09AF807464FF071
:1069E0000408C6EBC60000EB06112C48801C00EB27
:1069F00041008078284BDA1908F101016B1C0090E6
:106A000098B229A300F084F80746601C84B2042CD5
:106A100086DB2CE004984079012813D1A9F101000C
:106A20001F4909680978884204DC00201C4909686C
:106A3000087018E01A4800680078401C1849096876
:106A4000087010E016480068007828B9A9F1010024
:106A500013490968087006E0114800680078401E74
:106A60000F490968087000BF05B0BDE8F08F00BF8E
:106A70000948F9F781FE87B239460748FFF74EFC0F
:106A800007E0BAF1100F04D1BBF1010F00D100BF34
:106A9000EAE700BFE8E70000F8860020FC060020D7
:106AA0008802002025730000256400002DE9F041D4
:106AB00004460D4617460026032C12D1012D02D0A4
:106AC000022D02D100E002E001E0BDE8F08100BF4C
:106AD0000E48F9F751FE86B231460C48FFF71EFC0E
:106AE00012E0102C10D1012D02D0022D02D100E0B5
:106AF00001E000E0E9E700BF0448F9F73DFE86B297
:106B000031460248FFF70AFC00BFDEE7F8860020A6
:106B10000FB42DE9FC470746884615464FF48071AF
:106B20001B48F9F78DFE0EA801904FF480711848AC
:106B3000019B0D9AF9F78EFC0FFA80F9B9F1FF3F2E
:106B400002D0B9F5807F09DD0020019011A0F9F78E
:106B50009BFC0020BDE8FC075DF814FB0C48434695
:106B60003A4610A100902846F9F79AFC2846F9F712
:106B700003FE86B2002404E0FF2031196854601C33
:106B800084B2032CF8DB00200190F01C80B2E1E716
:106B9000F88E00204C656E677468205245454F5250
:106BA000000000007425645F25642E7478743D2213
:106BB00025732200FCF7F6FCFEF7A0F9FDF7FAFFBB
:106BC000FDF7A4FFFEF7ECF8FEF706F9FEF720F953
:106BD000FEF7A2F8FEF7C2F8FEF736F9FEF750F915
:106BE000FEF796FD01E0FEF7C1FDFCE770B5034638
:106BF0000C4603E014F8015B03F8015B151EA2F1DB
:106C00000102F7D170BD30B502464FF6FF7012E0B9
:106C100012F8014B6040002308E000F0010424B1A9
:106C20004AF2010484EA600000E040101C465D1C4A
:106C3000ABB2082CF1DB0C1EA1F10105A9B2E7D122
:106C400030BD00B97047002141610161C16000BFE2
:106C5000F8E770B504460D460CB9002070BDE06839
:106C600008B90020FAE745B1D4E90006236903FB1F
:106C7000060132462846FFF7B9FF2069401CA1688B
:106C800090FBF1F201FB12002061E068401EE06021
:106C90000120E3E770B504460D460CB9002070BD35
:106CA000D4E90210884201D10020F8E745B1D4E9C7
:106CB0000016636903FB061032462946FFF796FF6C
:106CC0006069401CA16890FBF1F201FB1200606159
:106CD000E068401CE0600120E1E770B504460D4625
:106CE0000CB9002070BDD4E90210884204DA2946AC
:106CF0002046FFF7CFFFF5E745B1D4E900166369F9
:106D000003FB061032462946FFF770FF6069401CFE
:106D1000A16890FBF1F201FB120060612069401C48
:106D2000A16890FBF1F201FB120020610120D9E77C
:106D300070477047704770477047000010B50249B0
:106D40004868804710BD0000A80000207047000080
:106D500010B50548C16C88470448C16C8847044891
:106D6000C16C884710BD000068010020B8010020F8
:106D70000802002010B500290AD00878002807D0A2
:106D800005487844FBF720F9002801D0002010BD09
:106D90000248784410BD0000F6010000EE0100003A
:106DA00010B500290AD00878002807D00548784493
:106DB000FBF70AF9002801D0002010BD02487844F2
:106DC00010BD0000E6010000DE0100004FF0407041
:106DD000E1EE100A7047FAF7E1B8FAF715BA0006C3
:106DE000101600061016000000000000000001024E
:106DF0000304060708090000000001020304040060
:106E00000008000000000000000200010000100067
:106E100000000000000000003031323334353637D6
:106E200038394142434445464030580030313233CE
:106E300034353637383961626364656640307800CE
:106E400030313233343536373839616263646566E0
:106E50007870003031323334353637383941424377
:106E60004445465850003A7474003A7474003A74B9
:106E70007400000002400000000000A000000000BC
:106E800005400000000000C8000000000C400000A9
:106E90000000409C00000000194000000020BCBE23
:106EA0000000000034400000BFC91B8E0000000439
:106EB000B5400000504BCFD06607E2CF0100000084
:106EC0006C4100003E8251AADFEEA73401000000B1
:106ED000D9420000DCB5A0E23A301F97FFFFFFFF68
:106EE000B4450000FD25A0C8E9A3C14FFFFFFFFF87
:106EF000FF3F00000000008000000000FF3F000096
:106F0000000000800000000056312E30000000001C
:106F1000313135323030000031393230300000004C
:106F20003537363030000000393630300000000090
:106F30003438303000000000434F4D310000000075
:106F4000434F4D3200000000434F4D33000000001E
:106F5000434F4D3400000000A470000800000020E2
:106F600098020000C4010008F47100089802002093
:106F7000C0940000200200081C0000004300000034
:106F8000F8FFFFFF0C0000000E0000000F000000E3
:106F90002E0000001001000043000000F8FFFFFF7A
:106FA000004040404040404040404141414141401C
:106FB00040404040404040404040404040404040D1
:106FC0004005020202020202020202020202020260
:106FD0000220202020202020202020020202020265
:106FE00002029090909090901010101010101010BD
:106FF00010101010101010101010101002020202C9
:10700000020288888888888808080808080808080C
:107010000808080808080808080808080202020208
:107020004000000000000000000000000000000020
:107030000000000000000000000000000000000050
:107040000000000000000000000000000000000040
:107050000000000000000000000000000000000030
:107060000000000000000000000000000000000020
:107070000000000000000000000000000000000010
:107080000000000000000000000000000000000000
:1070900000000000000000000000000000000000F0
:1070A0000000000041321042011324F413086F0065
:1070B0000A120856302E3030312E303A0128135142
:1070C0006D22081203320A3A330C120732323A4D5B
:1070D0000C120B32643A310C120D32C83A370C12D2
:1070E000111AF43D3A3D0C121323E8033A350C1201
:1070F0001723D0073A390CA11381571B08950413A5
:10710000055823088C1420F35A1408095B1B08F156
:10711000081AEF041AB014100E0D0E0F0C0B0A090A
:107120000807040302011B0605101608090A0B0CC8
:107130001F01020304050656211AD9401AED041A4C
:10714000CD04012013D1591B087D041A55041AC916
:10715000041AEC6413C8112A20F4E3B80B0B148052
:107160001D180B14382918191514208C031420BC71
:10717000051B205C0421120113F0341420A840ECFC
:1071800020B80B2E611A5BF0134D5C1B08B1041A7A
:107190007B0C1A2508411AC10C1A38501AD050130A
:1071A0007C061B201C04295013604C0C102018581E
:1071B000502B080220091C501A50501A485013FC3A
:1071C000041B209C04295013D0630C3520886FA029
:1071D000126F1B0840041A48041A50041A30041A8B
:1071E00028041A18041A20041A100481139D675BDE
:0471F0000880A481EE
:040000050800018965
:00000001FF
